:100000000C941D180C943A180C943A180C943A1845
:100010000C943A180C943A180C943A180C943A1818
:100020000C943A180C943A180C943A180C943A1808
:100030000C943A180C943A180C943A180C943A18F8
:100040000C943A180C943A180C943A180C943A18E8
:100050000C943A180C943A180C943A180C943A18D8
:100060000C943A180C943A1805A84CCDB2D44EB959
:100070003836A9020C50B9918688083CA6AAAA2A4B
:10008000BE000000803F0664EC1B3C04BC163E3BF7
:10009000E5B93CC93C37C29E5A3D660498083EEA21
:1000A00069AAAA3E000000803F2E2E2E676C65696B
:1000B0006368202020202020202020202020006491
:1000C0006572206A65747A74207765677363726FEE
:1000D0006C6C7400497267656E6465696E20546566
:1000E0007874005472616E73706172656E742C2046
:1000F00052756E64652025640074616E00636F73D1
:100100000073696E00756E74656E3B20463D255820
:100110000054696D657320766F6E206C696E6B7329
:100120003B20463D256400257500417269616C20C5
:10013000766F6E207265636874733B20463D004F96
:100140007269656E7420463D2558007777772E7466
:10015000752D6368656D6E69747A2E64652F7E797E
:1001600067753A202558004D696E692D46617262A7
:10017000646973706C61792D4269626C696F74682F
:10018000656B0000001FF800F8E0071F00E0FF03A8
:10019000060500E007E0FF807F00F810801F00FFE9
:1001A00007FFFF080C205F000000000000000000B7
:1001B000000000000020202020202000200000005F
:1001C000285050000000000000000000002828FC1B
:1001D0002850FC50500000002078A8A0603028A8CB
:1001E000F02000000048A8B0502834544800000017
:1001F0000020505078A8A8906C000000404080007B
:100200000000000000000000040810101010101082
:1002100008040000402010101010101020400000B2
:10022000000020A87070A8200000000000202020FE
:10023000F820202000000000000000000000000066
:100240004040800000000000F800000000000000B6
:100250000000000000000000400000000810101026
:10026000202040404080000000708888888888886E
:10027000700000000020602020202020700000007E
:100280000070888810204080F80000000070880806
:10029000300808887000000000103050509078102E
:1002A0001800000000F88080F00808887000000046
:1002B00000709080F08888887000000000F890102E
:1002C0002020202020000000007088887088888806
:1002D000700000000070888888780848700000006E
:1002E00000000020000000002000000000000000CE
:1002F00020000000202000000408102040201008EA
:1003000004000000000000F80000F80000000000F9
:100310004020100804081020400000000070888869
:10032000102020002000000000708898A8A8B88045
:10033000780000000020203050507848CC000000A9
:1003400000F0484870484848F00000000078888075
:10035000808080887000000000F048484848484885
:10036000F000000000F8485070504048F8000000CD
:1003700000F8485070504040E000000000384880CD
:10038000809C88483000000000CC484878484848A5
:10039000CC00000000F8202020202020F8000000E1
:1003A000007C10101010101090E0000000EC48507D
:1003B00060505048EC00000000E0404040404044A5
:1003C000FC00000000D8D8D8D8A8A8A8A800000031
:1003D00000DC486868585848E800000000708888C9
:1003E000888888887000000000F0484870404040CD
:1003F000E0000000007088888888E8987018000085
:1004000000F0484870504848EC00000000788880B0
:1004100060100888F000000000F8A82020202020AC
:100420007000000000CC48484848484830000000B0
:1004300000CC4848505030202000000000A8A8A858
:10044000705050505000000000D8505020205050A4
:10045000D800000000D8505020202020700000005C
:1004600000F8901020204048F8000000382020209C
:100470002020202020380000404040202010101074
:100480000800000070101010101010101070000004
:1004900020500000000000000000000000000000EC
:1004A000000000000000FC00200000000000000030
:1004B0000000000000000000304838483C00000008
:1004C00000C0404070484848700000000000000034
:1004D00038484040380000000018080838484848AC
:1004E0003C00000000000000304878403800000068
:1004F000001C202078202020780000000000000050
:100500003C4830407844380000C04040704848487B
:10051000EC0000000020000060202020700000009F
:1005200000100000301010101010E00000C040401B
:100530005C507048EC00000000E0202020202020CB
:10054000F800000000000000F0A8A8A8A800000023
:1005500000000000F0484848EC00000000000000E7
:10056000304848483000000000000000F04848488B
:100570007040E000000000003848484838081C007F
:1005800000000000D8604040E000000000000000D3
:1005900078403008780000000000202070202020E3
:1005A0001800000000000000D84848483C00000047
:1005B00000000000EC485030200000000000000067
:1005C000A8A870505000000000000000D850205033
:1005D000D800000000000000EC4850302020C0008F
:1005E0000000000078102020780000001810101083
:1005F00020101010101800101010101010101010F3
:1006000010101000602020201020202020600040CA
:10061000A4180000000000000000001010205F007F
:1006200000000000000000000000000000000000CA
:1006300000000000000000000000000000000000BA
:1006400000000007000F800F800F800F800F8007D1
:10065000000700000000000700070007000000007E
:10066000000E380E380E380E38063000000000003C
:10067000000000000000000000000000000000007A
:10068000000C300C300C307FFE7FFE0C300C300C38
:10069000300C307FFE7FFE0C300C300C3000000040
:1006A00000024002400FF81FF81A401A401FF00FD6
:1006B000F8025802581FF81FF002400240000000E4
:1006C00000000000000E100E300E7000E001C003AC
:1006D0008007000E700C7008700000000000000021
:1006E0000000000F001980198019800F000F080FFB
:1006F0009819F818F018E019F00F980000000000A1
:100700000000000700070007000E000000000000C6
:1007100000000000000000000000000000000000D9
:1007200000000000F001C0038007000E000E000E64
:10073000000E000700038001C000F0000000000070
:100740000000000F00038001C000E0007000700096
:1007500070007000E001C003800F00000000000086
:1007600000000001801188099007E007E03FFC3F8E
:10077000FC07E007E00990118801800000000000FC
:10078000000000000000000180018001800FF00FD8
:10079000F0018001800180000000000000000000E6
:1007A0000000000000000000000000000000000049
:1007B00000000000000700070007000E0000000016
:1007C000000000000000000000000000001FF81FF3
:1007D000F800000000000000000000000000000021
:1007E0000000000000000000000000000000000009
:1007F00000000000000700070007000000000000E4
:1008000000000000020006000E001C00380070000E
:10081000E001C0038007000E001C00000000000083
:100820000000000FF01C381C781CF81CF81DB81DC7
:10083000B81F381F381E381C380FF00000000000A9
:100840000000000180018003801F801F800380035F
:100850008003800380038003801FF00000000000FD
:100860000000000FE01C701C380038007000E00130
:10087000C0038007000E381C381FF800000000007D
:100880000000000FE01C701C380038007003C0032B
:10089000C0007000381C381C700FE0000000000021
:1008A00000000000E001E003E006E00CE018E01FBB
:1008B000F81FF800E000E000E003F800000000008E
:1008C0000000001FF81C001C001C001C001FE01F83
:1008D000F0007800381C381C700FE00000000000A9
:1008E00000000003E007000E001C001C001FF01FAA
:1008F000F81C381C381C381C380FF00000000000B1
:100900000000001FFC1C1C1C1C1C1C001C003800D0
:100910007000E001C003800380038000000000003D
:100920000000000FF01C381C381C381F3807E00787
:10093000E01CF81C381C381C380FF00000000000C8
:100940000000000FF01C381C381C381C381FF80F32
:10095000F800380038007000E007C0000000000018
:1009600000000000000000038003800380000000FE
:1009700000038003800380000000000000000000EE
:1009800000000000000000038003800380000000DE
:1009900000038003800380070000000000000000C7
:1009A00000007000E001C0038007000E001C001C66
:1009B000000E000700038001C000E000700000008E
:1009C0000000000000000000003FFC3FFC000000B1
:1009D000003FFC3FFC0000000000000000000000A1
:1009E000001C000E000700038001C000E000700042
:1009F0007000E001C0038007000E001C0000000032
:100A00000003C00FF01E7818380038007000E001B5
:100A1000C001C00000000001C001C001C000000012
:100A2000000FF81C1C1C1C1C1C1C1C1CFC1CFC1C93
:100A3000FC1CFC1C001C001C001FF007F800000040
:100A400000000003C007E00E701C381C381C381C66
:100A5000381FF81C381C381C381C380000000000F7
:100A60000000001FF00E380E380E380E380FF00F51
:100A7000F00E380E380E380E381FF000000000005F
:100A800000000007F00E381C381C001C001C001C65
:100A9000001C001C001C380E3807F000000000008D
:100AA0000000001FE00E700E380E380E380E380EA3
:100AB000380E380E380E380E701FE00000000000AF
:100AC0000000001FF80E180E080E000E300FF00F79
:100AD000F00E300E000E080E181FF8000000000087
:100AE0000000001FF80E180E080E000E300FF00F59
:100AF000F00E300E000E000E001F0000000000007F
:100B000000000007F00E381C381C381C001C001CAC
:100B1000001CF81C381C380E3807F80000000000D4
:100B20000000001C701C701C701C701C701FF01FDB
:100B3000F01C701C701C701C701C70000000000009
:100B40000000000FE0038003800380038003800324
:100B50008003800380038003800FE000000000001A
:100B600000000001FC007000700070007000700058
:100B70007038703870387038700FE0000000000076
:100B80000000001E380E380E700EE00FC00F800FF0
:100B9000800FC00EE00E700E381E380000000000FE
:100BA0000000001F000E000E000E000E000E000ED2
:100BB000000E000E080E180E381FF800000000008E
:100BC0000000001C1C1E3C1F7C1FFC1FFC1DDC1CAD
:100BD0009C1C1C1C1C1C1C1C1C1C1C000000000061
:100BE0000000001C1C1C1C1E1C1F1C1F9C1DDC1C50
:100BF000FC1C7C1C3C1C1C1C1C1C1C000000000061
:100C000000000003E007F00E381C1C1C1C1C1C1C00
:100C10001C1C1C1C1C0E3807F003E0000000000028
:100C20000000001FF00E380E380E380E380FF00F8F
:100C3000F00E000E000E000E001F0000000000006D
:100C400000000003E00F780E381C1C1C1C1C1C1C30
:100C50001C1C7C1CFC0FF80FF8003800FC00000086
:100C60000000001FF00E380E380E380E380FF00F4F
:100C7000F00E700E380E380E381E380000000000DE
:100C80000000000FF01C381C381C381C000FE00757
:100C9000F000381C381C381C380FF0000000000031
:100CA0000000001FFC19CC11C401C001C001C0012B
:100CB000C001C001C001C001C007F0000000000079
:100CC0000000001C701C701C701C701C701C701CC0
:100CD000701C701C701C701C700FE0000000000085
:100CE0000000001C701C701C701C701C701C701CA0
:100CF000701C701C700EE007C00380000000000034
:100D00000000001C1C1C1C1C1C1C1C1C1C1C9C1CF7
:100D10009C1C9C0FF80FF807700770000000000083
:100D20000000001C701C701C700EE007C0038003E4
:100D30008007C00EE01C701C701C700000000000DA
:100D40000000001C701C701C701C701C700EE007F2
:100D5000C003800380038003800FE00000000000D8
:100D60000000001FF81C381838107000E001C003A4
:100D70008007000E081C181C381FF8000000000037
:100D800000000007F0070007000700070007000742
:100D900000070007000700070007F0000000000040
:100DA000000000100018001C000E00070003800166
:100DB000C000E000700038001C00070000000000C8
:100DC00000000007F00070007000700070007000FC
:100DD00070007000700070007007F00000000000EC
:100DE00000018003C007E00E701C38000000000006
:100DF00000000000000000000000000000000000F3
:100E000000000000000000000000000000000000E2
:100E100000000000000000000000007FFF7FFF00D6
:100E20000000001C001C000700070000000000007C
:100E300000000000000000000000000000000000B2
:100E400000000000000000000000000FE000700043
:100E5000700FF01C701C701C700FD8000000000098
:100E60000000001E000E000E000E000FF00E380EE7
:100E7000380E380E380E380E381BF0000000000017
:100E800000000000000000000000000FE01C701CCB
:100E9000701C001C001C701C700FE00000000000A3
:100EA00000000000F80070007000700FF01C701C53
:100EB000701C701C701C701C700FD80000000000AB
:100EC00000000000000000000000000FE01C701C8B
:100ED000701FF01C001C701C700FE0000000000070
:100EE00000000003E007700770070007001FE01F05
:100EF000E007000700070007001FC0000000000017
:100F000000000000000000000000000FD81C701C52
:100F1000701C701C700FF007F000701C700FE00068
:100F20000000001E000E000E000E000EF00F380F25
:100F3000380E380E380E380E381E3800000000000B
:100F400000000001C001C001C000000FC001C001CD
:100F5000C001C001C001C001C00FF80000000000C6
:100F6000000000007000700070000003F0007000CE
:100F70007000700070007000701C700CF007E000D2
:100F80000000001E000E000E000E000E380E700E47
:100F9000E00FC00EE00E700E381E3800000000009A
:100FA0000000000FC001C001C001C001C001C001AC
:100FB000C001C001C001C001C00FF8000000000066
:100FC00000000000000000000000001FF81C9C1C36
:100FD0009C1C9C1C9C1C9C1C9C1C9C0000000000DD
:100FE00000000000000000000000001FE01C701C5A
:100FF000701C701C701C701C701C700000000000C5
:1010000000000000000000000000000FE01C701C49
:10101000701C701C701C701C700FE0000000000041
:1010200000000000000000000000001BF00E380E61
:10103000380E380E380E380FF00E000E001F00006C
:1010400000000000000000000000001FB038E03881
:10105000E038E038E038E01FE000E000E001F000B8
:1010600000000000000000000000001EF00FF80F5C
:10107000380E000E000E000E001F000000000000E1
:1010800000000000000000000000000FE01C301C09
:10109000300F8003E0187018700FE00000000000AF
:1010A00000000000000100030007001FF007000718
:1010B00000070007000770077003E0000000000051
:1010C00000000000000000000000001C701C701CEC
:1010D000701C701C701C701C700FD8000000000089
:1010E00000000000000000000000001C701C701CCC
:1010F000701C701C700EE007C00380000000000030
:1011000000000000000000000000001C1C1C1C1C53
:101110001C1C9C1C9C0FF80770077000000000004E
:1011200000000000000000000000001CE01CE00FB8
:10113000C0078007800FC01CE01CE000000000001A
:1011400000000000000000000000000E380E380E05
:10115000380E380E3807F003E000E001C01F8000B1
:1011600000000000000000000000001FE018E01177
:10117000C0038007000E201C601FE000000000007C
:1011800000000001F803800380038007001C001C9E
:1011900000070003800380038001F80000000000C6
:1011A0000001C001C001C001C001C001C001C001F7
:1011B000C001C001C001C001C001C001C0000000E9
:1011C0000000001F8001C001C001C000E000380025
:1011D0003800E001C001C001C01F80000000000015
:1011E0000000001F1C3B9C39DC38F80000000000A8
:1011F00000000000000000000000000000000020CF
:1012000032300A000000000000000000FFFE000174
:10121000FFFF0003FFFF8001FFFF600CFFFEF01ED9
:101220000001F83F0001F83F0001F83F0001F83FDE
:101230000001F83F0001F83F0001F83F0001F83FCE
:101240000001F83F0001F83F0001F83F0001F83FBE
:101250000001F83F0001F83E000078380000182037
:101260000000080000000020000000380000183EC8
:101270000000783F0001F83F0001F83F0001F83F0F
:101280000001F83F0001F83F0001F83F0001F83F7E
:101290000001F83F0001F83F0001F83F0001F83F6E
:1012A0000001F83F0001F83F0001F81E0000F00CBB
:1012B000FFFE6001FFFF0003FFFF8001FFFF000052
:1012C000FFFE000000000000000000000000000021
:1012D000000000000000000000000000000000000E
:1012E000000060000000F0000001F8000001F800BC
:1012F0000001F8000001F8000001F8000001F8000A
:101300000001F8000001F8000001F8000001F800F9
:101310000001F8000001F8000001F8000001F800E9
:101320000000780000001800000008000000000025
:101330000000000000001800000078000001F80024
:101340000001F8000001F8000001F8000001F800B9
:101350000001F8000001F8000001F8000001F800A9
:101360000001F8000001F8000001F8000001F80099
:101370000001F8000000F000000060000000000024
:10138000000000000000000000000000000000005D
:10139000000000000000000000000000FFFE00014F
:1013A000FFFF0003FFFF8001FFFF6000FFFEF00072
:1013B0000001F8000001F8000001F8000001F80049
:1013C0000001F8000001F8000001F8000001F80039
:1013D0000001F8000001F8000001F8000001F80029
:1013E0000001F8000001F80000007801FFFE18037A
:1013F000FFFF880FFFFFE027FFFFC039FFFF003E20
:101400000000003F0000003F0000003F0000003FE0
:101410000000003F0000003F0000003F0000003FD0
:101420000000003F0000003F0000003F0000003FC0
:101430000000003F0000003F0000001E0000000C04
:10144000FFFE0001FFFF0003FFFF8001FFFF000020
:10145000FFFE00000000000000000000000000008F
:1014600000000000FFFE0001FFFF0003FFFF8001FE
:10147000FFFF6000FFFEF0000001F8000001F8002F
:101480000001F8000001F8000001F8000001F80078
:101490000001F8000001F8000001F8000001F80068
:1014A0000001F8000001F8000001F8000001F80058
:1014B00000007801FFFE1803FFFF880FFFFFE00721
:1014C000FFFFC001FFFF1800000078000001F800D6
:1014D0000001F8000001F8000001F8000001F80028
:1014E0000001F8000001F8000001F8000001F80018
:1014F0000001F8000001F8000001F8000001F80008
:101500000001F8000000F000FFFE6001FFFF000393
:10151000FFFF8001FFFF0000FFFE00000000000051
:1015200000000000000000000000000000000000BB
:1015300000000000000000000000600C0000F01E31
:101540000001F83F0001F83F0001F83F0001F83FBB
:101550000001F83F0001F83F0001F83F0001F83FAB
:101560000001F83F0001F83F0001F83F0001F83F9B
:101570000001F83F0001F83E00007839FFFE182313
:10158000FFFF880FFFFFE007FFFFC001FFFF18000C
:10159000000078000001F8000001F8000001F800E8
:1015A0000001F8000001F8000001F8000001F80057
:1015B0000001F8000001F8000001F8000001F80047
:1015C0000001F8000001F8000001F8000000F00040
:1015D00000006000000000000000000000000000AB
:1015E00000000000000000000000000000000000FB
:1015F00000000000FFFE0001FFFF0003FFFF80016D
:10160000FFFF000CFFFE001E0000003F0000003F37
:101610000000003F0000003F0000003F0000003FCE
:101620000000003F0000003F0000003F0000003FBE
:101630000000003F0000003F0000003F0000003EAF
:1016400000000039FFFE0023FFFF800FFFFFE007CF
:10165000FFFFC001FFFF1800000078000001F80044
:101660000001F8000001F8000001F8000001F80096
:101670000001F8000001F8000001F8000001F80086
:101680000001F8000001F8000001F8000001F80076
:101690000001F8000000F000FFFE6001FFFF000302
:1016A000FFFF8001FFFF0000FFFE000000000000C0
:1016B000000000000000000000000000FFFE00012C
:1016C000FFFF0003FFFF8001FFFF000CFFFE001E75
:1016D0000000003F0000003F0000003F0000003F0E
:1016E0000000003F0000003F0000003F0000003FFE
:1016F0000000003F0000003F0000003F0000003FEE
:101700000000003F0000003E00000039FFFE002303
:10171000FFFF800FFFFFE027FFFFC039FFFF183EEC
:101720000000783F0001F83F0001F83F0001F83F5A
:101730000001F83F0001F83F0001F83F0001F83FC9
:101740000001F83F0001F83F0001F83F0001F83FB9
:101750000001F83F0001F83F0001F81E0000F00C06
:10176000FFFE6001FFFF0003FFFF8001FFFF00009D
:10177000FFFE00000000000000000000000000006C
:1017800000000000FFFE0001FFFF0003FFFF8001DB
:10179000FFFF6000FFFEF0000001F8000001F8000C
:1017A0000001F8000001F8000001F8000001F80055
:1017B0000001F8000001F8000001F8000001F80045
:1017C0000001F8000001F8000001F8000001F80035
:1017D0000000780000001800000008000000000071
:1017E0000000000000001800000078000001F80070
:1017F0000001F8000001F8000001F8000001F80005
:101800000001F8000001F8000001F8000001F800F4
:101810000001F8000001F8000001F8000001F800E4
:101820000001F8000000F00000006000000000006F
:1018300000000000000000000000000000000000A8
:10184000000000000000000000000000FFFE00019A
:10185000FFFF0003FFFF8001FFFF600CFFFEF01E93
:101860000001F83F0001F83F0001F83F0001F83F98
:101870000001F83F0001F83F0001F83F0001F83F88
:101880000001F83F0001F83F0001F83F0001F83F78
:101890000001F83F0001F83E00007839FFFE1823F0
:1018A000FFFF880FFFFFE027FFFFC039FFFF183E53
:1018B0000000783F0001F83F0001F83F0001F83FC9
:1018C0000001F83F0001F83F0001F83F0001F83F38
:1018D0000001F83F0001F83F0001F83F0001F83F28
:1018E0000001F83F0001F83F0001F81E0000F00C75
:1018F000FFFE6001FFFF0003FFFF8001FFFF00000C
:10190000FFFE0000000000000000000000000000DA
:1019100000000000FFFE0001FFFF0003FFFF800149
:10192000FFFF600CFFFEF01E0001F83F0001F83FD2
:101930000001F83F0001F83F0001F83F0001F83FC7
:101940000001F83F0001F83F0001F83F0001F83FB7
:101950000001F83F0001F83F0001F83F0001F83EA8
:1019600000007839FFFE1823FFFF880FFFFFE00714
:10197000FFFFC001FFFF1800000078000001F80021
:101980000001F8000001F8000001F8000001F80073
:101990000001F8000001F8000001F8000001F80063
:1019A0000001F8000001F8000001F8000001F80053
:1019B0000001F8000000F000FFFE6001FFFF0003DF
:1019C000FFFF8001FFFF0000FFFE0000000000009D
:1019D000000000FD10205F2163B60822632111661C
:1019E000666666661166668D9889970885A69898DA
:1019F0008886C868161164625666611550A06566CF
:101A00005251844424200600000008000000000019
:101A100000000000000000000000000000000000C6
:101A200000000000000000000000000000000000B6
:101A300000000000000000000000000000000000A6
:101A40000000000000000000000000000000000096
:101A50000000000000000000000000000000000086
:101A6000000000000000000000224221E1C20381CA
:101A70000904000000238040F070043F0E1FC38162
:101A8000C0000000001C01F80207F81F0FE0FF9FD4
:101A9000E0F0404809012010048083C1FC0783F86E
:101AA0001F1FF40480A040A0280BFDE38400100059
:101AB00040000080060040448080000000000000DC
:101AC0000000000000000006B0000224222922408D
:101AD000441109F0000002440C110880C2011008F2
:101AE000442200000000022060605040820881080B
:101AF00001001084048090220180CC0842102084D0
:101B00002042081040480A0A090441009208A00037
:101B100080040000080080040008080000000000A5
:101B2000000008000000000000888000224224928B
:101B30002404411084000000482142090814202098
:101B4000808824100000000041080105040440487A
:101B500008801002044048090420180CA0881101D4
:101B6000102202404104044110A108841011108A7F
:101B7000000000400000800800400080800000005D
:101B800000000000800000000000088800022444DB
:101B9000482280441108A04000048224008082442E
:101BA00002001082412200800804110E905040482B
:101BB000008048010040040480908201414A0900ED
:101BC000901201202400104044110A1088220111B3
:101BD00009100003C5C0E0E871E3A5C44829738B70
:101BE0008385C0E9679E850610C183FC888000203C
:101BF0001FF482280280204A040000482040081870
:101C0000247C2E010444100071FC7001111888849A
:101C10000880080480100400404809102014149023
:101C20009009012012022001040441111105014014
:101C30002110910000426211118888466244849804
:101C4000C4C444621198848850610A28208888009E
:101C5000020044381C803002040040000482040169
:101C6000070444231020384100180000C0222088B7
:101C7000887F0800804FF1004007FC80930201221A
:101C80004889009022012041C010404221111020BB
:101C90001404110A080008241202090488242448A4
:101CA000890848482412090808848929148410885E
:101CB0008E20200440E013850020403F80008820D3
:101CC00040100884012082044230020000020424F3
:101CD00008888408800804801FC43E4048095020BA
:101CE0001224889009FC2013F803810404220912AD
:101CF00005008041088000000E412020904882426B
:101D000044909084848241209080884892914441FC
:101D100008891C020044090144888204004000082C
:101D2000820402005040120820821D00180000C0EA
:101D3000824109FC4048008048010040240480980A
:101D40008201144849009002012100041040422001
:101D5000A0A0880808108800000724120209FC8847
:101D600024244B090848482412090788845145084F
:101D70004423086000201FF09024485020400403B2
:101D8000C08820404005FE0120820820100071FC20
:101D90007008241090440480080480100402404914
:101DA0000904201144829009002012080041040413
:101DB000140A0A08808101088000008241202090D6
:101DC00008824244C890848482412090048845144B
:101DD00051428408880002008849024482020400BB
:101DE000400008820408104044120840824100006C
:101DF000800800824111044044048088010020448E
:101E000004909042011448288110011B2084041082
:101E1000404140A0A10408101088000008241202CC
:101E20000904882424488908484824120900488461
:101E30005145142840888000000882A04444502066
:101E400040000001044041018804221104044220A2
:101E50000000000000223220240820881080100199
:101E6000084049090220108481842100086204206E
:101E70008102080804042020820104800000866298
:101E8000111188884642448490848444621190846D
:101E900088C2082222880888000200881C0438387A
:101EA00081080000805038043F870041C0E040387E
:101EB0001C2200000000811DC2027F01F0FE0FF90C
:101EC000000F04048F1013F90848083C10007B2011
:101ED00021F0101F0080404401087FD04800000717
:101EE000A5C0E0E87083A424482908484385C0E9D8
:101EF000078E7420824111FC888000000000800061
:101F00000000108000080000000000000000000039
:101F10000000002000000000080080000000000019
:101F200000000000000000000000000000000000B1
:101F30000000000000000000000000000100800020
:101F4000000000000000000200040000000000404B
:101F50000080000000000001000888000000000070
:101F600000000001080000800000000000000000E8
:101F700000000000020000000000603000000000CF
:101F80000000000000000000000000000000000051
:101F90000000000000000000000000000000100829
:101FA00000000000000000000840004000000000A9
:101FB00004000800000000000010008880000000FD
:101FC0000000000000090000000000000000000008
:101FD000000000000000000000000001FC00000004
:101FE00000000000000000000000000000000000F1
:101FF00000000000000000000000000000000001E0
:10200000C3807FC0000000000000780008000000CE
:1020100000004000800000000000060006B000FD47
:1020200012205F3275D61C3386322266666666667B
:10203000218858AEA98AB83AA4D8BAB88AA9FABAF7
:10204000383275536757651661B176775362A66665
:102050006560070000011040000000000300400020
:10206000000004000000000000000000000000006C
:1020700000000000007C00000000000000000000E4
:102080000000000000000000000000000000000050
:10209000000000000000000000000000000001E857
:1020A0003C00003000C000006000E003019980C0E7
:1020B0000000000000000000000000000000000020
:1020C000623000003198223E3C0403C06090080258
:1020D0000000009E060783C030780E7F1F0F0000AF
:1020E00000000001E030600C1FF00F2FF87FEFFCC4
:1020F0000F27EFFF7FF9EFC1E01FC1F07C3FC03C2D
:102100001FE01E9FFFF9FF87FDF1FF8FFC79FFB1F4
:1021100001860003003800001C002600E033703800
:10212000000000000000000010000000000000009F
:10213000184300000633088D6CC100C40C210D60EB
:102140004000002663C1399C061F070FC6333000CC
:10215000008004004608060180C3061C61830460F9
:10216000861C3061830C10600E071C0830C18C186F
:1021700060C6063318CC0860230C18C0860220669F
:10218000103120002003000001800C000C00060329
:102190000000000000000000060000000000000039
:1021A0000608300000C66111A5984018818C307077
:1021B000080000048418432181C2018208C6C300BC
:1021C00000E000700C621940581861808C18608C17
:1021D0001180860C3061840C01C0E1C10C0C30C64A
:1021E000061861824309810C0860820C2060841803
:1021F000C20624000000600000300180018000C0A1
:10220000600000000000000000C0000000000000AE
:1022100000C10600001889FFB43310031021020E1C
:1022200001000000B0C3006030586060021898667A
:1022300060600001818C86E40B030C2011818C41CD
:10224000882010C1860C3101802C2C3C2180C618BE
:1022500080430C3040603020C1061840C80620067C
:102260001840C84000078DC0F0761CFC3C37199917
:10227000ECDCE370786E0766CEBFCEF3FBDFDFE702
:102280007F1820C000031104438662006C0460665E
:10229000B02000002618600C0C131F0B8041A30C0B
:1022A000CC701FF80E01118C8260618C0030318877
:1022B000310C001830C1864030058585846018C314
:1022C000300C6183800C06041840C7101A00C4004B
:1022D000C3041908000199CC3319C6460CF73773AB
:1022E00011BCE6F3199E619DEA3318CC26313118F2
:1022F00048C30418000040019830CC9E063C0C0CEA
:1023000010FFE00004C30C0103C2607398081C6155
:10231000801000000020466110460FE18006063F55
:1023200007E183F3FE1830F006009130988C031813
:10233000C6018C603C0180C0818818A201800D001C
:102340003060832100003330CC26198CC18CC666E6
:10235000643318CC661986619842631984C6234396
:10236000081860830000080022030F2661E2018143
:102370008200800F00986180401C8C06618206C636
:102380003001C0000038108C2210C1863000C0C659
:1023900020C4301860C3061B00C01326119180634F
:1023A000F0C031F001E0301810310196401800C043
:1023B0000C0C1068100000E61980C33F983198CCCF
:1023C000CD0663198CC330CC330E0C63190CE83086
:1023D0003206181031C201001FF87008CCCC403012
:1023E00030001001E0230C301801A1804C30418CEA
:1023F0007C00060FFC1804130C43F8306600181814
:10240000C41886030C1860C330180264C21A300C5A
:1024100060180633000E060302034034D00580180E
:102420000301810C0000006CC330186603033319EC
:1024300099E0CC63319866198660F18C6321AD0216
:1024400006418402014E400000880B0219B0D006FC
:102450000600020000046186020037F80986103188
:1024600081800038001C0082611041860CC003038B
:10247000180300E061830C18630302471843C60188
:102480000C0300863040C0C0604068068A013003FB
:1024900000C03021800000199866030CC0607C6386
:1024A0003336198C66330CC330CC07318C6435A0BD
:1024B000E070606040C870000011096083361C0045
:1024C000C0C0004000008420C08406060130C2065F
:1024D00030600000800400004C621030C18C046049
:1024E000C302600C0C3061830C306048E308386034
:1024F00061803030C30C18180C08060061C043001E
:102500006018160430000003330CE2619C4C100C80
:10251000666663318CC66198661984263187039C90
:10252000260E0C0608300000C00441AC1066E3889B
:1025300018180008180320CC183FB180CC43304055
:10254000E61833000000000309BC86071860C10CC0
:1025500030608C00E1860C3341830C110861030666
:102560001830030C1831C60300C200C00C30103004
:102570000C0606C04600000066630F8679F183F9F9
:102580008CCCC6663198C663986730C4D678E06351
:102590000860C308C10600001800881F04078F8E5A
:1025A000010200000380640F0FCFE7C019F03C1058
:1025B0000F1C0670000000006119E3E1FFF80FC76F
:1025C000F83FF7E007E3F7FFB0FCFFFEF93FF82024
:1025D0003C1F803E0FC3A781F80F800800820F0FB9
:1025E00087E1FF9808C0000007E7C0E0761CFC3FC9
:1025F000FBFDBDFFEF7FBC786E076F171C760804EC
:10260000239E10FF1820C000000000008000000082
:102610000030C000001000000000000000000000BA
:102620000000000200000000001000800000000018
:10263000000000000000000000000000000000009A
:102640000000000380000000000000000000000007
:102650000000000300180000000000000000000857
:1026600010003000000000000C000C000000000012
:102670000000020003041800000000000000000039
:102680000002100000040000000000000000000034
:102690000000000080000000000200200000000098
:1026A000000000000000000000000000000000002A
:1026B0000000000018000000000000000000000002
:1026C00000000000600300000000000000000002A5
:1026D00002000600000000000180018000000000F0
:1026E0000000008000608300000000000000000087
:1026F00000002400000100000000000000000000B5
:102700000000000020000000000020080000000081
:1027100000000000000000000000000000000000B9
:102720000000000001C000000000000000000000E8
:10273000000000000C00600000000000000000002D
:1027400060800080000000000030003000000000C9
:10275000000000F0000610C00000000000000000B3
:102760000000030000000000000000000000000066
:102770000000000000000000000003020000000054
:102780000000000000000000000000000000000049
:1027900000000000000E000000000000000000002B
:1027A0000000000001E03C01FF800000000000008C
:1027B00007E0002000000000000F000F00000000F4
:1027C0000000001C0000623000000000000000005B
:1027D00000000000000000000000000000000000F9
:1027E00000000000000000000000001F800000004A
:1027F00000000000000000000000000000000000D9
:1028000000000000000000000000000000000000C8
:1028100000000000000000000000000000000000B8
:1028200000000000000000000000000000000000A8
:1028300000000000000000000000FFFFFFFFFFFF9E
:10284000FFFFFFFFFFFFFFFFFFFFFFFFFFFFFFFF98
:10285000FFFF3CE7D39CF39C14A5F39C518C75AD12
:10286000FFFFFFFFFFFFFFFFFFFFFFFFFFFFFFFF78
:10287000FFFFFFFFFFFFFFFFFFFFFFFFFFFFFFFF68
:10288000FFFFFFFFFFFFFFFFFFFFFFFFFFFFFFFF58
:102890007DEFEB5AEF7BD39CB294B294B294284272
:1028A000EF7BFFFFFFFFFFFFFFFFFFFFFFFFFFFFCC
:1028B000FFFFFFFFFFFFFFFFFFFFFFFFFFFFFFFF28
:1028C000FFFFFFFFFFFFFFFFFFFFFFFFDFFFFFFF38
:1028D000F39CE3180C63494A694A694A8A52494A97
:1028E000000038C6FFFFDFFFFFFFFFFFFFFFFFFF16
:1028F000FFFFFFFFFFFFFFFFFFFFFFFFFFFFFFFFE8
:10290000FFFFFFFFFFFFFFFFFFFFFFFFDFFFFFFFF7
:102910006D6B00002000A2108210410841084108A0
:1029200000000C63FFFFFFFFFFFFFFFFFFFFFFFF44
:10293000FFFFFFFFFFFFFFFFFFFFFFFFFFFFFFFFA7
:10294000FFFFFFFFFFFFFFFFFFFFFFFFDFFFFFFFB7
:102950008A52284210840000610855ADD7BDA210EC
:1029600000004529BEF7FFFFFFFFFFFFFFFFFFFF4E
:10297000FFFFFFFFFFFFFFFFFFFFFFFFFFFFFFFF67
:10298000FFFFFFFFFFFFFFFFFFFFFFFFDFFFFFFF77
:10299000CB5A718C5DE726218B525DE7DBDECF7B66
:1029A0000000E3183CE7FFFFFFFFFFFFFFFFFFFF13
:1029B000FFFFFFFFFFFFFFFFFFFFFFFFFFFFFFFF27
:1029C000FFFFFFFFFFFFFFFFFFFFFFFFDFFFFFFF37
:1029D0006D6B4A4A2A6BE78B8AA4096B8A4A318459
:1029E000000004213CE7FFFFFFFFFFFFFFFFFFFFA9
:1029F000FFFFFFFFFFFFFFFFFFFFFFFFFFFFFFFFE7
:102A0000FFFFFFFFFFFFFFFFFFFFFFFFDFFFFFFFF6
:102A10006E6B04526ADEF7FFF8FFACD5AABC665AAB
:102A200000008210FBDEFFFFFFFFFFFFFFFFFFFF45
:102A3000FFFFFFFFFFFFFFFFFFFFFFFFFFFFFFFFA6
:102A4000FFFFFFFFFFFFFFFFFFFFFFFFDFFFFFFFB6
:102A5000108C40C5EDFF2CFFECFECCFE66FE6082C4
:102A60000000000096B5FFFFDFFFFFFFFFFFFFFF45
:102A7000FFFFFFFFFFFFFFFFFFFFFFFFFFFFFFFF66
:102A8000FFFFFFFFFFFFFFFFFFFFFFFFDFFFFFFF76
:102A9000B394259C20FF40FEA0FDC0FC24F56A8372
:102AA000000000000C63FFFFDFFFFFFFFFFFFFFFE1
:102AB000FFFFFFFFFFFFFFFFFFFFFFFFFFFFFFFF26
:102AC000FFFFFFFFFFFFFFFFFFFFFFFFDFFFFFFF36
:102AD0000C63B49413FF83FD23F5CFE59EF71DE748
:102AE000610800006108DBDEFFFFFFFFFFFFFFFF63
:102AF000FFFFFFFFFFFFFFFFFFFFFFFFFFFFFFFFE6
:102B0000FFFFFFFFFFFFFFFFFFFFDFFFFFFF59CECC
:102B100041089AD6FFFF7DFF7DF7FFFFFFFFFFFF14
:102B2000AE7300000000694AFFFFDFFFFFFFFFFFF9
:102B3000FFFFFFFFFFFFFFFFFFFFFFFFFFFFFFFFA5
:102B4000FFFFFFFFFFFFFFFFFFFFFFFF9EF7A2104A
:102B50001084FFFFDFFFFFFFFFFFFFFFDFFFFFFF2F
:102B600059CE0000000000009294FFFFDFFFFFFF3E
:102B7000FFFFFFFFFFFFFFFFFFFFFFFFFFFFFFFF65
:102B8000FFFFFFFFFFFFFFFFFFFFFFFFAA52200035
:102B9000BEF7FFFFFFFFFFFFFFFFDFFFDFFFBEF717
:102BA000DFFF863100002000410879CEFFFFDFFF04
:102BB000FFFFFFFFFFFFFFFFFFFFFFFFFFFFFFFF25
:102BC000FFFFFFFFFFFFDFFFFFFF38C60000AA5235
:102BD000FFFFDFFFFFFFFFFFDFFFDFFFBEF79EF717
:102BE000FFFFF39C000041080000E739DFFFFFFF13
:102BF000FFFFFFFFFFFFFFFFFFFFFFFFFFFFFFFFE5
:102C0000FFFFFFFFFFFFFFFFFFFFCB5A0000F7BDF5
:102C1000FFFFDFFFFFFFDFFFDFFFBEF7BEF79EF71F
:102C20009EF77DEF863100006108000055ADFFFF83
:102C3000DFFFFFFFFFFFFFFFFFFFFFFFFFFFFFFFC4
:102C4000FFFFFFFFFFFFFFFF3CE76108494AFFFF6F
:102C5000FFFFFFFFDFFFDFFFDFFFBEF79EF77DEF28
:102C60005DEFDFFF1084000082100000E739DFFF16
:102C7000FFFFFFFFFFFFFFFFFFFFFFFFFFFFFFFF64
:102C8000FFFFFFFFDFFFFFFFB294000096B5FFFFDD
:102C9000DFFFDFFFDFFFDFFFBEF79EF77DEF7DEF9A
:102CA0003CE79EF755AD6108A2106108410859CE76
:102CB000FFFFFFFFFFFFFFFFFFFFFFFFFFFFFFFF24
:102CC000FFFFFFFFFFFF9EF78531A2101CE7FFFF0C
:102CD000DFFFDFFFDFFFBEF79EF77DEF7DEF5DEFEC
:102CE0003CE75DEFF7BDC318C318C3180000718C33
:102CF000FFFFDFFFFFFFFFFFFFFFFFFFFFFFFFFF04
:102D0000FFFFDFFFFFFFB2940000E739BEF7FFFFD0
:102D1000DFFFDFFFBEF79EF77DEF7DEF5DEF3CE766
:102D20001CE71CE718C6E318A210A21020004D6B88
:102D3000FFFFFFFFFFFFFFFFFFFFFFFFFFFFFFFFA3
:102D4000FFFFDFFFFFFF518CE038274AFFFFDFFF67
:102D5000BEF7BEF79EF77DEF7DEF5DEF3CE71CE72A
:102D6000FBDE1DDFF8BDC739CB5A8A52A3108F7323
:102D7000FFFFFFFFFFFFFFFFFFFFFFFFFFFFFFFF63
:102D8000FFFFFFFFFFFF6CDD2BFE45BC13A5FFFF20
:102D9000BEF79EF79EF77DEF5DEF3CE71CE7FBDE9D
:102DA000DCD68EDDE4B3242165294529C12011B587
:102DB000FFFFFFFFFFFFFFFFFFFFFFFFFFFFFFFF23
:102DC000FFFF7CF7CFE50BF69BFF54FF028BF07BF8
:102DD000DFFF9EF75DEF5DEF3CE71CE7FBDEDBDE30
:102DE0007ACE89EDADDD42080000000069AC6BDDF4
:102DF000BFEFFFFFFFFFFFFFFFFFFFFFFFFFBEFF74
:102E0000CBE5C9ED4BFE14FFF3FE35FF8DFEC1513E
:102E10004E633CE75DEF3CE71CE7FBDEDBDEDBD629
:102E200059CE8BE598FF4FBD888B90CDB7FFE8CC8E
:102E30003DE7FFFFFFFFFFFFFFFFFFFFFFFF3BEF50
:102E400083F530FF11FFCFFEEFFECFFE30FF46DDF2
:102E500003298E6B7DEF1CE7FBDEDBDEBAD69AD64C
:102E600059CEAAE511FF53FF73FF33FF12FF6CFE2B
:102E7000ADDD9EF7FFFFFFFFFFFFFFFFFFFF9EF7A8
:102E8000C5EDCBFECCFECCFEECFECBFECCFEEAFECE
:102E9000E59B32843CE7DBDEDBDEBAD69AD6DBDEAE
:102EA000F3A447D52EFFCDFECEFEEEFEEEFE10FFC4
:102EB000ABFEA8E57DEFFFFFFFFFFFFFFFFF9EF7E3
:102EC00003F6A2FEC7FEC7FEA4FE81FE61FEA4FEBD
:102ED00043FE33DE5EE71CE7FBDEDBDE58CE728CA2
:102EE0004752E4ED0AFFCAFEC9FE84FE83FEE7FEF8
:102EF000A3FE43B49BD6FFFFFFFFFFFFFFFF5BF77F
:102F000060FE00FFC0FEC0FEA0FEA0FEC0FEA0FE50
:102F1000E0FEC1E5929414A5D39C10840B63294272
:102F2000E86A80FEC1FEC1FEA0FEA0FEE0FE80DDDC
:102F3000E89B97B5DFFFFFFFFFFFFFFFFFFF9EF757
:102F400089D500E6A0FE00FF40FF40FF00FF00FF24
:102F500020FFC0FE67522942484A494A89524A42E4
:102F6000467B20FFE0FEE0FE20FFE0FEA5B4929C41
:102F7000FDDEFFFFFFFFFFFFFFFFFFFFFFFFFFFF84
:102F80001DE7B6BD30B50BBD65CD60EE40FFA0FFBF
:102F900080FF03BD108414A534A575AD96B555A565
:102FA0008F9CC0F6A0FFA0FFE0F649A4B8B5FFFFD4
:102FB000FFFFFFFFFFFFFFFFFFFFFFFFFFFFFFFF21
:102FC000FFFFFFFFFFFF7FEF9CD695BD4CBDC6CD39
:102FD000E8B435ADBFF7FFFFFFFFFFFFFFFFFFFFC7
:102FE000BFF7D0CDC6CDA7CD8DA47BCEFFFFFFFF11
:102FF000FFFFFFFFFFFFFFFFFFFFFFFFFFFFFFFFE1
:10300000FFFFFFFFFFFFFFFFFFFFFFFF1FDF9AB57F
:10301000DABDFFFFFFFFDFFFFFFFFFFFDFFFDFFF87
:10302000FFFF7FEF9AB559AD1DDFFFFFDFFFFFFF09
:10303000FFFFFFFFFFFFFFFFFFFF11241FBECFEFCA
:10304000D8E0DEBFCDBF11E0A0E0B1E0E4E3FCE6F4
:1030500002C005900D92A430B107D9F713E0A4E0A7
:10306000B1E001C01D92A030B107E1F70E94BA1B88
:103070000C94F42F0C940000CF92DF92EF92FF9209
:103080000F931F937C0169010E945A25C701B60165
:10309000A8010E94282A1F910F91FF90EF90DF90C6
:1030A000CF9008950F931F93CF93DF9360913C01CE
:1030B00070913D0140913E0150913F0184E091E0CB
:1030C0000E9442258FE190E090932B0180932A018A
:1030D00010922D0110922C01809129018D7F8093F7
:1030E000290100913E0110913F0144275527401BC3
:1030F000510B84E091E060E070E020E030E00E945D
:103100003C1820913C0130913D0166277727621BD6
:10311000730B84E091E040E050E000E010E00E949A
:103120003C18C0E6DFEF84E091E0BE0142E050E0F1
:103130009E0100E010E00E943C182A96CA3AD10590
:1031400091F7C0E6DFEF84E091E06EEF7FEFAE0134
:1031500020E030E08E010E943C182A96CA3AD10540
:1031600091F7DF91CF911F910F9108950F931F93C6
:10317000CF93DF93EC0110920D0110920C0110928D
:103180000F0110920E018091280180FD29C000E4FA
:1031900011E020EF30E0235030400151104084E036
:1031A00091E062E070E04FE050E00E94A424D093F0
:1031B0002D01C0932C01809129018D7F80932901DD
:1031C00084E091E0BE010E94052CC095D095D0937B
:1031D0002B01C0932A01DF91CF911F910F91089588
:1031E00000EF10E020E431E0D6CF0F931F938C0165
:1031F0000E945A25C8010E9408281F910F91089526
:10320000CF92DF92EF92FF920F931F937C0169019F
:103210000E945A25F70185A1806185A3C701B601E7
:10322000A8010E948525C7010E94A525C701029615
:103230000E94A5251F910F91FF90EF90DF90CF90F6
:103240000895EF92FF920F931F937C010E94001943
:10325000C7010E94EB281F910F91FF90EF900895F6
:10326000FF920F931F930E94E42FF82E0E94E42FE9
:10327000082F0E94E42F3F2D20E02070387F10E0BF
:1032800095E0000F111F9A95E1F7007E1770202B33
:10329000312B86958695869590E0282B392B309397
:1032A0002B0120932A011F910F91FF9008950F93F6
:1032B0001F938C010E94E42FB8010E947D351F915D
:1032C0000F91089584E391E00E94712F0895AF92C9
:1032D000BF92CF92DF92EF92FF920F931F93CF9303
:1032E000DF93C0E8D2E08BE090E00E945719059789
:1032F0008993999382E0C039D807A9F760E9C62E6F
:1033000062E0D62EF60138968091280190E09C016B
:103310002170307080FD03C080EF90E002C080E437
:1033200091E0959587959093910280939002909368
:103330009902809398022115310519F480EF90E0ED
:1033400002C080E491E0909395028093940221154D
:10335000310519F480E491E002C080EF90E095958A
:103360008795909397028093960290939F02809303
:103370009E02232B19F480E491E002C080EF90E0DC
:1033800093838283AA24BB2480912C0190912D01E8
:1033900090932B0180932A010894A11CB11C8501F4
:1033A0000370107034E0000F111F3A95E1F70057D9
:1033B0001D4F84E091E0B80144E050E00E94CB2A28
:1033C000C0E8D2E0780148815981F601808191817D
:1033D000480F591FF701518340838A819B81F60171
:1033E00022813381820F931FF7019383828357FDDC
:1033F0000CC08091280180FD03C080EF90E002C0E6
:1034000080E491E0481759075CF085E090E00E9465
:10341000571928813981821B930B029799838883DE
:10342000F7012281338137FD0CC08091280180FD96
:1034300003C080E491E002C080EF90E028173907D4
:103440005CF085E090E00E9457192A813B81821B45
:10345000930B02979B838A83249684E090E0E80E86
:10346000F91EC80ED91E92E0C039D90709F0ABCFBA
:10347000F50125E0F695E7952A95E1F7EE70F070F5
:10348000ED56FE4F8591949190932B0180932A01E4
:1034900084E091E0B80144E050E00E94CB2A80E251
:1034A0009EE40197F1F70E946219882339F46801BC
:1034B000E0E0AE16E1E0BE0609F066CFDF91CF9105
:1034C0001F910F91FF90EF90DF90CF90BF90AF9042
:1034D00008950F931F93CF93DF93EC0110920D018A
:1034E00010920C0110920F0110920E0184E091E0F5
:1034F00060E070EE40E050EE20E030E200E010E2EC
:103500000E94A4248FEF9FEF90932B0180932A01B8
:1035100084E091E067E070E047E050E027E030E0D1
:103520000E948D2B0EC00E946219882369F488EED8
:1035300093E0E0E9F1E03197F1F70197D1F7C45654
:10354000D0401C161D067CF380EE9FEF90932B015C
:1035500080932A0184E091E067E070E047E050E06A
:1035600027E030E00E948D2B8091280180FDCEC0A5
:1035700000E411E020EF30E02350304001511040D2
:1035800084E091E062E070E04FE050E00E94A4240B
:10359000B7C084E391E060ED0E94762FA0E0B0E038
:1035A000BC01CD0120EF30E040E050E00E945E35EC
:1035B000BC0188279927EB0184E391E060E90E9430
:1035C000762FA0E0B0E0BC01CD0120E431E040E086
:1035D00050E00E945E35BC01882799278B018091BD
:1035E0002801282F82FF06C08FE391E0AC01401B29
:1035F000510B8A0121FF06C08FEE90E0AC014C1BFD
:103600005D0BEA0120FF03C0C8018E01EC0180E0E0
:103610009EEF90932B0180932A0184E091E0BE01FC
:10362000A80124E130E00E948D2B8FE190E090937F
:103630002B0180932A0184E091E0BE01A80124E1DE
:1036400030E00E94182884E091E0BE01A80125E145
:1036500030E00E94182884E091E0BE01A80126E134
:1036600030E00E941828C436D1050CF041C0043661
:1036700011050CF03DC084E091E06BE176E00E9422
:10368000B12DBE0168507040A8014850504084E000
:1036900091E00E945A2582E08093290184E091E024
:1036A00060E50E94262C8CED95E0E0E9F1E0319791
:1036B000F1F70197D1F70E946219882309F58CED83
:1036C00095E0E0E9F1E03197F1F70197D1F78091CA
:1036D0002A0190912B012FE13EEF822793279093AF
:1036E0002B0180932A010E946219882351F208C09D
:1036F00080EA9FE0E0E9F1E03197F1F70197D1F737
:103700000E946219882309F044CF05C000EF10E041
:1037100020E431E031CFDF91CF911F910F910895D7
:10372000EF92FF920F931F93CF93DF937801C0E046
:10373000D0E016C00E94301980E491E00E94571931
:103740008C0180E491E00E945719AC0184E091E083
:10375000B8010E94F5180E946219882321F421966D
:10376000CE15DF053CF3DF91CF911F910F91FF90B4
:10377000EF900895AF92BF92CF92DF92EF92FF92B7
:103780000F931F93CF93DF9384E391E00E94562F12
:10379000E0913601F0913701E370F070E157FE4F90
:1037A000E49184E091E06E2F0E94CE268091280162
:1037B00080FD03C080EF90E002C080E491E0959529
:1037C000879590933D0180933C018091280180FD75
:1037D00003C080E491E002C080EF90E0959587956A
:1037E00090933F0180933E0188E190EC90932D01EE
:1037F00080932C01809129018D7F8093290184E0A1
:1038000091E068E170EC0E94052C80EE9FEF9093B0
:103810002B0180932A0184E091E067E070E047E0AB
:1038200050E027E030E00E948D2B10922B01109287
:103830002A0184E091E063EA71E00E94B12D84E006
:1038400091E062E170E041E050E00E945A2584E09E
:1038500091E067E671E00E94282D80EF9FEF909342
:103860002B0180932A018091280180FD03C040E450
:1038700051E002C040EF50E0C4E0D1E0809131015E
:10388000992787FD9095481B590B42505040CE0117
:1038900068E070E00E945A2500D000D000D0EDB75B
:1038A000FEB73196ADB7BEB71296DC93CE931197A3
:1038B0008BE491E093838283809128018483158235
:1038C0000E94F42DEDB7FEB736960FB6F894FEBF02
:1038D0000FBEEDBF8FEF9FEF0E94B618CE0168E3D9
:1038E00070E048E350E020E830E000E810E00E949B
:1038F0000019CE0160E070E040E850E00E941B2F0C
:10390000CE016BE176E00E94B12DCE0164E170E062
:1039100044E150E00E945A2500D000D000D0EDB71D
:10392000FEB73196ADB7BEB71296DC93CE93119722
:103930008FE391E0938382838091280184831582B1
:103940000E94F42DEDB7FEB736960FB6F894FEBF81
:103950000FBEEDBFCE0163ED79E10E94B12DCE0126
:1039600064E170E04CED50E00E945A2580912801FE
:103970008770886680932801CE016AE271E00E9418
:10398000282DCE016FEF71E10E94B12D80912901A8
:10399000806180932901CE0160EF7FEF40E050E02D
:1039A0000E945A2500D000D000D0EDB7FEB7319666
:1039B000ADB7BEB71296DC93CE93119787E291E034
:1039C0009383828380913801909139019583848318
:1039D0000E94F42DEDB7FEB736960FB6F894FEBFF1
:1039E0000FBEEDBFCE016FE170E20E94B12DCE019E
:1039F0006CED70E044E150E00E945A25809128016E
:103A0000877088658093280100D000D000D0EDB782
:103A1000FEB73196ADB7BEB71296DC93CE93119731
:103A200081E191E09383828380913A0190913B01FF
:103A3000958384830E94F42DEDB7FEB736960FB6BA
:103A4000F894FEBF0FBEEDBFCE016BE176E00E94A1
:103A5000B12DCE016CED70E04CED50E00E945A2586
:103A600020912801277020632093280100D000D0E6
:103A700000D0EDB7FEB73196ADB7BEB71296DC9366
:103A8000CE93119785E091E09383828324831582FE
:103A90000E94F42DEDB7FEB736960FB6F894FEBF30
:103AA0000FBEEDBF88EB9BE00E94691ACE0163EA6E
:103AB00071E00E94B12D80912801877080932801C8
:103AC00020913C0130913D0180913E0190913F0158
:103AD0008217930734F4CE016FED70E044E150E0BB
:103AE00005C0CE0164E170E04CED50E00E9442253B
:103AF00080E098EF90932B0180932A0184E091E07D
:103B000060E070E040E050E024E130E004E110E0EB
:103B10000E94211980EE97E090932B0180932A0157
:103B200084E091E064E170E044E150E028E230E0BC
:103B300008E210E00E9421198FE190E090932B01A0
:103B400080932A0184E091E06EE170E046E450E069
:103B50002CE330E00CE310E00E94211988EB9BE09D
:103B60000E94691A10920D0110920C0110920F011F
:103B700010920E010E94671980E090E00E94B61832
:103B80000E94521884E091E063ED79E10E94B12D2A
:103B900082E0809329018FEF97E090932B0180932F
:103BA0002A0164E070E080913C0190913D01681B26
:103BB000790B40E150E080913E0190913F01481B1C
:103BC000590B84E091E00E945A2584E091E061E085
:103BD00071E00E94282D80913C0190913D01CC27FD
:103BE000DD27C81BD90B2CC0BE01882777FD809527
:103BF000982F0E94E83027ED33EA40E95FE30E9406
:103C0000AD3123EC35EF48E450E40E94AD3120E0C3
:103C100030E044E353EC0E944D300E94103220E02B
:103C200030E040EA52E40E94AD310E94B5309B0181
:103C3000AC0184E091E0BE01A9010E94F518219633
:103C400020913C0130913D012C173D076CF680E03E
:103C500098EF90932B0180932A0164E070E0621B3F
:103C6000730B40E250E080913E0190913F01481B70
:103C7000590B84E091E00E945A2584E091E06DEFB9
:103C800070E00E94282D80913C0190913D01CC274D
:103C9000DD27C81BD90B2CC0BE01882777FD809576
:103CA000982F0E94E83027ED33EA40E95FE30E9455
:103CB000AD3123EC35EF48E450E40E94AD3120E013
:103CC00030E044E353E40E944D300E944A3020E04B
:103CD00030E040EA52EC0E94AD310E94B5309B01C9
:103CE000AC0184E091E0BE01A9010E94F518219683
:103CF00020913C0130913D012C173D076CF680EE80
:103D00009FEF90932B0180932A0164E070E0621B87
:103D1000730B40E350E080913E0190913F01481BBE
:103D2000590B84E091E00E945A2584E091E069EF0C
:103D300070E00E94282D60913C0170913D017095CA
:103D400061957F4F84E091E040E050E00E945A2569
:103D500080913C0190913D01CC27DD27C81BD90BF8
:103D60002CC0BE01882777FD8095982F0E94E830EF
:103D700027ED33EA40E95FE30E94AD3123EC35EFF4
:103D800048E450E40E94AD3120E030E044E353ECDD
:103D90000E944D300E94163220E030E040E252E4B2
:103DA0000E94AD310E94B5309B01AC0184E091E0EE
:103DB000BE01A9010E94282A219680913C01909180
:103DC0003D018C179D076CF688EB9BE00E94691AF9
:103DD00088EB9BE00E94691A80E090E00E94B61890
:103DE0000E945218C0E0D0E001E0C02ED12C27C0C4
:103DF000F0E4CF16F1E0DF0614F1C03AD10531F05E
:103E0000FE01E05CFE4F8081882339F48FE190E071
:103E100090932B0180932A0104C010922B011092E1
:103E20002A01BE01605A7040FE01E05CFE4F4081F5
:103E3000552747FD509584E091E00E94F5188FEFDB
:103E400097E090932B0180932A01B601882777FD94
:103E50008095982F0E94E8302DEC3CEC4CE85FE315
:103E60000E94AD3123EC35EF48E450E40E94AD31BF
:103E700020E030E044E353E40E944D300E941032D1
:103E80007B018C01C6016AE67FEF0E947D35615897
:103E90007F4F882777FD8095982F0E94E8309B01FF
:103EA000AC01C801B7010E94AD310E94B5308B0151
:103EB0009C01FE01E05CFE4F6083C05AD04084E06C
:103EC00091E0BE01A8010E94F518CF55DF4F81E0B7
:103ED000C034D80711F4C0E0D0E00E9462198823F2
:103EE00049F40894C11CD11C90E0C91692E3D9068C
:103EF00009F07ECF88EE93E00E94691A80E090E09E
:103F00000E94B61815E8A12E11E0B12E7501CAE580
:103F1000D0E0F7018591949190932B0180932A0131
:103F200084E091E0BE01A897AE012CE330E00CE301
:103F300010E00E942119A2E0B0E0EA0EFB1EEC9610
:103F4000BFE8EB16B1E0FB0621F788EB9BE00E948F
:103F5000691A80E090E00E94B618B6EFCB2EBFEF52
:103F6000DB2ECE0CDF1CCAEAD0E0F60185919491DD
:103F700090932B0180932A014CED50E04C1B5D0B7C
:103F800008E111E00C1B1D0B84E091E0BE01EC96F2
:103F90009E01A3E0EA2EF12C0E94FE2AE2E0F0E06E
:103FA000CE0EDF1EC055D040FFE8CF16F1E0DF0691
:103FB000E1F688EB9BE00E94691A80E090E00E94A5
:103FC000B618C8E7D0E0F5018591949190932B0144
:103FD00080932A0184E091E0BE01A897AE012EE112
:103FE00030E00E948D2B82E090E0A80EB91EEC9686
:103FF0009FE8A91691E0B90631F788EB9BE00E9493
:10400000691A80E090E00E94B61880E098EF9093E3
:104010002B0180932A01E0902201F09023018091EE
:104020001E0190911F01E81AF90AC0E0D0E018C003
:1040300060911C0170911D0140911E0150911F0162
:104040004C0F5D1F9E01220F331F260F371F00915B
:1040500022011091230184E091E00E943C182596F2
:10406000CE15DF052CF3E70119C000911E01109158
:104070001F016091200170912101AE01400F511F7D
:104080009E01220F331F80911C0190911D01280F6A
:10409000391F84E091E00E943C1825971C161D06EC
:1040A00024F38FEF97E090932B0180932A01E7018F
:1040B00019C000911E0110911F0160911C017091A7
:1040C0001D01AE01400F511FCE01880F991F209195
:1040D000200130912101281B390B84E091E00E94DE
:1040E0003C1825971C161D0624F3C0E0D0E019C02B
:1040F000609120017091210140911E0150911F019A
:104100004C0F5D1FCE01880F991F9B01281B390B97
:10411000009122011091230184E091E00E943C185B
:104120002596CE15DF0524F38FEF9FEF90932D0199
:1041300080932C0182E08093290160913C01709171
:104140003D016051704040913E0150913F0140510E
:10415000504084E091E020E230E000E210E00E9474
:10416000001984E091E06AE378E240E250E00E94C6
:104170001B2F88EB9BE00E94691A80E090E00E9470
:10418000B618C0E0D0E00E94301980E491E00E94AF
:1041900057197C0180E491E00E9457198C018EE14F
:1041A00090E00E9457199C0184E091E0B701A801BA
:1041B0000E9418282196C436D10529F788EB9BE088
:1041C0000E94691A80E090E00E94B618C0E0D0E03A
:1041D0000E94301980E491E00E9457195C0180E44C
:1041E00091E00E9457196C0180E491E00E945719F8
:1041F0007C0180E491E00E9457198C0184E091E0F9
:10420000B501A60197010E94DC292196C436D1058B
:10421000F9F688EB9BE00E94691A80E090E00E942A
:10422000B618C0E0D0E00E94301980E491E00E940E
:1042300057195C0180E491E00E9457196C0180E4F9
:1042400091E00E9457197C0180E491E00E94571987
:104250008C0184E091E0B501A6019701B3E0EB2E5B
:10426000F12C0E9435292196C436D105E1F688EB60
:104270009BE00E94691A80E090E00E94B61800E07E
:1042800010E00E9430198091280180FD03C080EF6A
:1042900090E002C080E491E004970E945719EC017D
:1042A0008091280180FD03C080E491E002C080EF8E
:1042B00090E080970E9457192296AC01405F5F4FB3
:1042C00084E091E0BE010E945A258091280180FD82
:1042D00003C080EF90E002C080E491E004970E9468
:1042E0005719EC018091280180FD03C080E491E022
:1042F00002C080EF90E080970E9457192296AC018F
:10430000405F5F4F84E091E0BE010E94282A0E9436
:104310006219882339F40F5F1F4FA1E0043F1A0789
:1043200009F0AFCF84EF91E00E94691A80E090E03D
:104330000E94B6188091280180FD3FC100E411E081
:1043400020EF30E0A4E0CA2EA1E0DA2E2151304067
:1043500001511040C60160E170E040E150E00E9470
:10436000A42482E090E060E170E04CE351E021EDB4
:1043700030E000E117E20E94901B84EF91E00E9480
:10438000691A8FE190E00E94B6188FE190E4909353
:104390002B0180932A01C60168E770E044E950E0F0
:1043A0002EE030E00E948D2BA12CF8EFBF2EB092B2
:1043B0002B01A0922A01C6016FE070E04FE350E0AC
:1043C00023EE30E001E810E0E3E0EE2EF12C0E9455
:1043D000FE2A80EF97EC90932B0180932A01C6016F
:1043E00060E170E04CE850E00E945A2582E0809342
:1043F000290120913601309137012F5F3F4F3093D3
:1044000037012093360100D000D000D0EDB7FEB7C1
:104410003196ADB7BEB71296DC92CE92119783EE6D
:1044200090E093838283358324830E94F42DEDB73B
:10443000FEB736960FB6F894FEBF0FBEEDBFC601AD
:1044400060E170E040E450E021EE30E00FE710E082
:104450000E94A424B0922D01A0922C0180912901E8
:104460008D7F8093290180913101992787FD909557
:1044700090933F0180933E01C0E0D0E07BC08FEF7E
:104480009FEF90932B0180932A0104E011E040E418
:1044900050E04C1B5D0BC80160E170E00E945A25A2
:1044A00000D000D0ADB7BEB712961C930E931197F3
:1044B00084ED90E014969C938E9313970E94F42DB4
:1044C0000F900F900F900F9040913E0150913F013F
:1044D000405C5F4F4C1B5D0BC80160E170E00E94C7
:1044E0005A2500D000D0EDB7FEB7128301838FEBC1
:1044F00090E0948383830E94F42D40913E0150917B
:104500003F010F900F900F900F90440F551F405C8C
:104510005F4F4C1B5D0BC80160E170E00E945A25A3
:10452000C80169EA70E00E94282D80E098EF90931E
:104530002B0180932A0180913E0190913F01AC01B3
:10454000440F551F405C5F4F480F591F4C1B5D0BBC
:10455000C80160E170E022ED30E001E010E00E946F
:10456000211980E29EE40197F1F70E9462198823E5
:1045700071F4219620913E0130913F01C901880FCD
:10458000991F820F931F8C179D070CF078CF809195
:10459000280180FD05C020E431E040EF50E004C078
:1045A00020EF30E040E451E080E090E060E070E037
:1045B00008E813E10E94901BE7C800EF10E020E438
:1045C00031E0C0CECF92DF92EF92FF920F931F9314
:1045D000DF93CF93CDB7DEB74BE0E42EF12CEC0E9A
:1045E000FD1EF701C190D1907F011092F40284E08A
:1045F0008093F50280ED92E060E070EE40E050EED6
:1046000020E030E200E010E20E94A4241092F702C1
:104610001092F6028FEF9FEF9093F9028093F802C9
:104620008091F5028D7F8093F50280ED92E06FE13D
:1046300070E20E94B12D80ED92E0B601A7010E94C8
:10464000D32D1092D1021092D0028091FD029927B1
:1046500087FD90952091D2023091D302820F931F53
:104660009093D3028093D2028353914024F010920E
:10467000D3021092D202CF91DF911F910F91FF9040
:10468000EF90DF90CF9008959BB94498449A8BB9EE
:104690004498449A089588B1886388B987B188633B
:1046A00087B98FEF8AB90895EF92FF920F931F9306
:1046B0007C018B0160E070E020E030E0CB01BA01CA
:1046C000A90198010E945E359B01AC01611571053D
:1046D00081059105C9F0762FBB27A52F942F832F35
:1046E000682FCA01AA27BB2721116F5F61118F5F55
:1046F000FBB84498449AEBB84498449A7150C1F777
:104700006150B1F78150A1F71F910F91FF90EF9089
:1047100008950F931F938B01459890E00E944423C6
:10472000459AC8010E9444231F910F910895439810
:10473000439A08954398439A08954398439A089555
:104740004398439A08954398439A08954398439A07
:104750000895FF920F931F938A01F22E80E2822721
:104760000E94892381E28F25B8010E948923459800
:1047700082E290E00E944423459A1F910F91FF909E
:104780000895FF920F931F93CF93DF93EC01162FA1
:104790000CA1017067FF22C0002361F0862F90E01A
:1047A0009C01220F331F2470959587958270282BCA
:1047B000197F122B612F70E067707070802F90E06E
:1047C0006827792723E0660F771F2A95E1F780E3B2
:1047D00090E16827792783E00E948923F12E16FF54
:1047E0001CC0102F110F6C857D8580E581270E94EC
:1047F00089236E857F8582E581270E9489236889C8
:10480000798981E581270E9489236A897B8983E5EB
:1048100081270E948923012F0695F4FE0AC0688132
:1048200079814A815B8120E0011121E0CE010E9463
:10483000A923DF91CF911F910F91FF900895EF92DF
:10484000FF920F931F93CF93DF93FC01EA0104A122
:10485000102F169516951695212F30E08689978989
:10486000A489B589A9014270507010FF1EC07B0158
:10487000E81AF90ABE016A1B7B0BDB01452B29F004
:10488000628973896E0D7F1D04C0668577856E19F8
:104890007F0922FF05C0408951894A0F5B1F20C054
:1048A000448555854A1B5B0B1BC07B01EA1AFB0A3A
:1048B000C81BD90B452B29F0608971896E0D7F1DAE
:1048C00004C0648575856E197F0922FF05C0428981
:1048D00053894C0F5D1F04C0468557854C1B5D0BEB
:1048E000212F30E0802F90E0282739272170307069
:1048F000CF010E94A923DF91CF911F910F91FF90CB
:10490000EF900895FC0184A186FF0FC026813781B6
:1049100087FF07C082819381880F991F821B930BA9
:1049200001C0C9019383828308952481358187FF63
:1049300007C080819181880F991F821B930B01C052
:10494000C9019183808308950F931F93CF93DF93C1
:10495000FC01E901A5A1A4FF0EC020853185620FED
:10496000731F82859385480F591FC20FD31F080FED
:10497000191FAF7EA5A384A180FD24C020E431E0EF
:1049800080EF90E077FF02C060E070E0718F608F91
:1049900057FF02C040E050E0538F428F0197C81785
:1049A000D9070CF4CE01958F848FC90101970817A0
:1049B00019070CF4C801978F868FDF91CF911F9153
:1049C0000F91089520EF30E080E491E0DBCFFC010F
:1049D000208D318D84859585A901481B590B11A225
:1049E00010A21416150624F43587248751A340A37A
:1049F000248D358D808991892817390714F4318BDE
:104A0000208B80899189019624853585821B930BA3
:104A1000958B848B20E0181619060CF421E0822F68
:104A20000895FC0120813181808D918D28173907EF
:104A3000A4F0848D958D821793077CF04281538179
:104A4000828D938D4817590744F020E0868D978D0D
:104A5000841795071CF021E001C020E0822F089503
:104A6000CF93DF93EC010E941125882341F0CE0102
:104A700060E30E94C1238EA19FA10E944423DF9185
:104A8000CF910895FC0125A124FF0FC08085918559
:104A9000860F971F9187808782859385840F951F46
:104AA000938782872F7E25A3089571876087538718
:104AB00042870895FC0125A124FF0FC080819181C8
:104AC000860F971F9183808382819381840F951F26
:104AD000938382832F7E25A3089580859185860FF9
:104AE000971F9183808382859385840F951F93837D
:104AF000828308950F931F938C010E945A25C80149
:104B00000E9430251F910F910895FC0125A124FFDB
:104B10000FC080819181860F971F95838483828146
:104B20009381840F951F978386832F7E25A30895F5
:104B300080859185860F971F9583848382859385D1
:104B4000840F951F978386830895FC012481358106
:104B500080819181A901481B590B57FF0DC03587F2
:104B6000248788279927841B950B958B848B21504C
:104B70003040280F391F09C095878487558B448B97
:104B80009C0121503040240F351F318B208B08951C
:104B90000F931F938C010E94A525C80102960E94C5
:104BA000A5251F910F910895FC01808D918D95870A
:104BB0008487828D938D97878687848D958D918B41
:104BC000808B868D978D938B828BCF0160EC0E94BA
:104BD000C12308952F923F925F926F927F928F929E
:104BE0009F92AF92BF92CF92DF92EF92FF920F937C
:104BF0001F93CF93DF93EC017B015A0189010E943F
:104C0000E724882309F4B5C0CE0102960E94E72468
:104C1000882309F4AEC028A139A14AA15BA18CA1C7
:104C2000682F70E0DB01A870B07083FF03C0CA0179
:104C3000A9019C01F901E00FF11F4A9DC0014B9DA4
:104C4000900D5A9D900D1124E80FF91F8C889D88B6
:104C5000CE88DF88AB2B19F0C60164014C018F01AF
:104C600093E0159507959A95E1F70E0D1F1D87E0C6
:104C7000E82EF12CEE22FF2215012818390843985E
:104C8000B3E075956795BA95E1F76770606FCE01EF
:104C90000E94C1236624F801449197012095309524
:104CA0002770307081E090E002C0880F991F2A952C
:104CB000E2F7782E542E54018DA1272D30E0452D9A
:104CC00050E081FF14C024233523232B19F46624DC
:104CD000639418C0662029F0CE01B501A6010E9498
:104CE0001F248EA19FA10E94442366240BC024236D
:104CF0003523232B19F08EA19FA102C088A599A569
:104D00000E9444230894E11CF11C0894A108B108F6
:104D1000A114B10499F0872D90E095958795782E90
:104D2000882351F60F5F1F4FF801849128EF3FEF62
:104D3000E20EF31E582EF0E87F2EBECF0894C10875
:104D4000D108C114D10489F09701220D331DC90186
:104D5000E3E095958795EA95E1F7080F191F77E04D
:104D6000E72EF12CE222F32296CFCE010E94D42529
:104D7000439ACE010E948224DF91CF911F910F911F
:104D8000FF90EF90DF90CF90BF90AF909F908F906B
:104D90007F906F905F903F902F9008950F931F9397
:104DA000CF93DF93EC016CA31DA260E070EE40E0B6
:104DB00050EE20E030E200E010E20E94A4241986C8
:104DC00018861B861A8688B1886388B987B188637C
:104DD00087B98FEF8AB9439885EE60EF78E70E9434
:104DE00089236CA170E07695762F66277795679575
:104DF0006070717081E00E94892382E060E072E05F
:104E00000E94892383E060E370E10E94892384E0AB
:104E100060E070E00E94892388E067E072E00E9411
:104E2000892389E060E070E00E9489238AE060E0E5
:104E300070E00E9489238CE060E070E00E9489238A
:104E40008DE060E070E00E9489238FE060E070E018
:104E50000E94892380E160E070E00E94892381E163
:104E600067E070E00E94892382E160E070E00E94C8
:104E7000892383E160E070E00E94892387E061E09C
:104E800070E00E94892380ED97E0E0E9F1E031973E
:104E9000F1F70197D1F780E160E976E10E9489237B
:104EA00081E167E272E00E94892384EF91E0E0E90A
:104EB000F1E03197F1F70197D1F782E16DE070E011
:104EC0000E94892384EF91E0E0E9F1E03197F1F766
:104ED0000197D1F783E160E072E10E94892389E2C2
:104EE0006AE070E00E9489238BE26DE070E00E942E
:104EF000892384EF91E0E0E9F1E03197F1F7019740
:104F0000D1F780E360E070E00E94892381E364E0F0
:104F100074E00E94892382E363E070E00E948923A9
:104F200085E365E074E00E94892386E368E078E029
:104F30000E94892387E367E074E00E94892388E365
:104F400063E073E00E94892389E367E077E00E94D1
:104F500089238CE364E075E00E9489238DE368E097
:104F600078E00E948923CE010E94D4258CA1782F5D
:104F70007295770F707E60E060707078776280E67F
:104F80000E94892381E661E070E00E9489238AE61D
:104F900060E070E00E94892380E860E070E00E9499
:104FA000892381E860E070E00E94892382E860E064
:104FB00070E00E94892383E860E070E00E9489230A
:104FC00084E860E070E00E94892385E860E070E09A
:104FD0000E94892380E960E170E00E94892382E9D0
:104FE00060E070E00E94892387E063E371E00E9443
:104FF0008923439A1FA21EA28FEF9FEF99A788A72C
:105000008DA18D7F8DA3DF91CF911F910F91089579
:1050100043980E943025439A08950F931F938C0163
:105020000E945A25C8010E9408281F910F910895D7
:105030002F923F924F925F926F927F928F929F92A8
:10504000AF92BF92CF92DF92EF92FF920F931F9396
:10505000DF93CF9300D000D000D0CDB7DEB79E83D2
:105060008D832B013A01890141E0242E312C221A33
:10507000330AC901880F991F22273327281B390BB0
:105080003A8329834398ED81FE8185A18F7E85A394
:10509000A801460D571D8D819E810E947A25A3018E
:1050A000401B510B8D819E81B2010E947A25B8016F
:1050B000640D751D8D819E81A3010E947A25B20128
:1050C000601B710B8D819E81A3010E947A2548018E
:1050D00021E030E03C832B83AA24BB245EC037FC54
:1050E0000AC008948108910889819A8102969A835E
:1050F0008983280E391E0894A11CB11CEB81FC8108
:105100003296FC83EB832E0E3F1E6501C40CD51C2A
:105110008401060D171D8D819E81B601A8010E9494
:105120007A257201EA18FB088D819E81B701A801DA
:105130000E947A258301081919098D819E81B60183
:10514000A8010E947A258D819E81B701A8010E9445
:105150007A256401C40CD51C8501060D171D8D81AF
:105160009E81B601A8010E947A257201E818F9080B
:105170008D819E81B701A8010E947A2583010A19B9
:105180001B098D819E81B601A8010E947A258D811F
:105190009E81B701A8010E947A25A814B9040CF4D5
:1051A0009ECF439A26960FB6F894DEBF0FBECDBFB2
:1051B000CF91DF911F910F91FF90EF90DF90CF90F3
:1051C000BF90AF909F908F907F906F905F904F9027
:1051D0003F902F900895CF93DF93EC010E94E72436
:1051E0008823B9F0CE0102960E94E724882389F033
:1051F0004398CE0160EF0E94C1236C897D894E895E
:105200005F898EA19FA10E945423CE010E94D425C4
:10521000439ADF91CF910895CF92DF92EF92FF9260
:105220000F931F937C0169010E945A25F70185A104
:10523000806185A3C701B601A8010E948525C70129
:105240000E94C825C7010E94EB281F910F91FF9073
:10525000EF90DF90CF9008950F931F9301E010E03F
:105260000E9421191F910F9108952F923F924F9202
:105270005F926F927F928F929F92AF92BF92CF92E6
:10528000DF92EF92FF920F931F93DF93CF9300D0A3
:1052900000D0CDB7DEB73C014B015C834B832901C5
:1052A00058012617370714F42B0149012B813C8143
:1052B000A216B30624F4C50159019C838B83120105
:1052C0002818390835E0231631040CF45EC0C501F6
:1052D000EB81FC818E1B9F0B9A83898305970CF4CD
:1052E00054C064010894C11CD11C8F010F5F1F4F73
:1052F000C301B601A8010E94F51872010894E108E3
:10530000F108C301B701A8010E94F51885010150F9
:105310001040C301B601A8010E94F518C301B701EE
:10532000A8010E94F51884010E5F1F4F6CEFE62E56
:105330006FEFF62EE20CF31CC301B8014B815C81C8
:1053400097010E942C29C301B801A50197010E9471
:105350002C2952E0E52EF12C2B813C81E20EF31E2C
:10536000C980DA808CEF9FEFC80ED91EC301B4014B
:10537000A70121E030E086010E942119C301B2019A
:10538000A70121E030E00E9421190F900F900F90AB
:105390000F90CF91DF911F910F91FF90EF90DF90D1
:1053A000CF90BF90AF909F908F907F906F905F90C5
:1053B0004F903F902F9008958F929F92AF92BF92FF
:1053C000CF92DF92EF92FF920F931F93CF93DF93D1
:1053D0004C01EB015A01690178012617370714F4D3
:1053E0006B01E901EA14FB0414F475015601F401A0
:1053F00085A18F7E85A386010C1B1D0BC401BE01F8
:10540000A50198010E942C29C401BE01A7019801A1
:105410000E942C29EA18FB08C401BE01A50121E065
:1054200030E087010E942119C401B601A50121E0E5
:1054300030E00E942119DF91CF911F910F91FF90D1
:10544000EF90DF90CF90BF90AF909F908F90089596
:10545000CF92DF92EF92FF920F931F93CF93DF9340
:10546000EC010E948525CE010E94C8256C897D89AA
:105470006115710579F48C859D85998B888B2DA19B
:1054800030E0217030708A899B89820F931F9B8B3B
:105490008A8B13C04E895F8941155105D1F48E85E1
:1054A0009F859B8B8A8B2DA130E02170307088897D
:1054B0009989820F931F998B888BCE010E94EB28CC
:1054C0008C819D81998388838E819F819B838A8330
:1054D00059C02C813D81888199812817390724F092
:1054E000F1E0CF2ED12C03C0CC24CA94DC2C2E8129
:1054F0003F818A819B812817390724F0E1E0EE2E55
:10550000F12C03C0EE24EA94FE2C8B01041B150B36
:10551000439823C0CE010E943025A801440F551F97
:105520002E893F89CA01820F931F1816190644F469
:10553000021B130B888199818C0D9D1D9983888393
:105540008C899D894817590744F4080F191F8A81CF
:105550009B818E0D9F1D9B838A83288139818C813D
:105560009D8128173907B1F62A813B818E819F8161
:105570002817390779F68DA180FF03C0CE010E945C
:105580003025439ADF91CF911F910F91FF90EF90BB
:10559000DF90CF900895CF92DF92EF92FF920F931A
:1055A0001F93CF93DF936C018B017A01FA0131973E
:1055B000EE0FFF1FEE0FFF1FE60FF71F60817181D7
:1055C000428153810E945A25E80100E010E00AC0A0
:1055D000688179814A815B81C6010E94282A0F5F18
:1055E0001F4F24960E151F059CF3DF91CF911F913D
:1055F0000F91FF90EF90DF90CF9008952F923F9200
:105600004F925F926F927F928F929F92AF92BF92D2
:10561000CF92DF92EF92FF920F931F93CF93DF937E
:105620002C016B014A01A90158012617370714F410
:10563000AB016901A814B9041CF4C50154014C0163
:105640003A016C187D0885E0681671040CF452C0AC
:10565000C50188199909853091050CF44BC01C01CE
:1056600035942794C0E0D0E0209721F0C130D105D7
:1056700061F513C086010E5F1F4F8CEFE82E8FEF90
:10568000F82EE60CF71CC201B801A40197010E9494
:105690002C29C201B801A50116C086010F5F1F4F5A
:1056A000BEEFEB2EBFEFFB2EE60CF71CA4014F5F05
:1056B0005F4FC201B80197010E942C29A5014150FA
:1056C0005040C201B80197010EC0AE01480D591DEE
:1056D000C201B60193010E942C29A5014C1B5D0B50
:1056E000C201B60193010E942C2921962C163D0679
:1056F0000CF0BACFDF91CF911F910F91FF90EF90F7
:10570000DF90CF90BF90AF909F908F907F906F90E1
:105710005F904F903F902F9008952F923F924F921D
:105720005F926F927F928F929F92AF92BF92CF9231
:10573000DF92EF92FF920F931F93CF93DF934C0171
:105740001B01FC0185A18F7E85A3CC24DD24C21A18
:10575000D30A229F2001239F500C329F500C11240A
:105760003601640E751E5A01AC18BD08E6012EC044
:10577000229FC001239F900D329F900D1124840F12
:10578000951F48165906B4F08901020D131D220F0A
:10579000331FEE24FF24E21AF30AC401B801A30167
:1057A00097010E942C29C401B801A50197010E940C
:1057B0002C2905C02F5F3F4F12161306CCF62196F9
:1057C0000894611C711C0894A108B1081C161D06E0
:1057D0004CF0CC9FA001CD9F500DDC9F500D1124AB
:1057E0009601EACFDF91CF911F910F91FF90EF903B
:1057F000DF90CF90BF90AF909F908F907F906F90F1
:105800005F904F903F902F9008950F931F93CF93E9
:10581000DF93EC018B0143980E94D4256C857D8534
:105820004E855F8520E08CA1811121E0CE010E9490
:10583000A923C80160EF70E040E451E00E945423C6
:10584000439ADF91CF911F910F910895BF92CF920C
:10585000DF92EF92FF920F931F93CF93DF93EC01B0
:10586000BDA1B2FF3EC06A30E1F58CA1982F96959C
:10587000969596959827892F829586958670892783
:10588000482F80FF17C08A859B859B838A838DA5BF
:105890002881398141FF06C0992787FD9095281BF3
:1058A000390B05C0992787FD9095280F391F39833B
:1058B0002883B1C088859985998388838DA52A819D
:1058C0003B8142FF06C0992787FD9095281B390B25
:1058D00005C0992787FD9095280F391F3B832A83A0
:1058E0009AC05EA5651750F0862F90E04FA5252F32
:1058F00030E0240F311D821793070CF06FE3651B16
:10590000562F6CA54DA5EAA4FBA416160CF43CC0BA
:10591000BFA400E010E0CC24DD24A0E072E031E080
:10592000F7010894E11CF11C9491292F2F70261B7C
:10593000872F8250851711F4A22F6801020F111DC5
:105940003B15A1F0892F90E0E4E095958795EA95C5
:10595000E1F78F70861B351711F4A82F6801080F27
:10596000111D7B1519F07E5F3E5FDACF8A2F9927D4
:1059700087FD9095909339018093380100933A0107
:1059800010933B016A2F28C0062F112707FD1095A1
:10599000095F1F4F087F802F90E073E095958795F2
:1059A0007A95E1F7242F332727FD3095F9018E9F53
:1059B00090018F9F300D9E9F300D1124852F90E018
:1059C000FC012E9FC0012F9F900D3E9F900D112432
:1059D000E80EF91ECC24DD248CA1982F83FF03C090
:1059E000842F462F682F94FD619595FD4195B061F8
:1059F000BDA3772767FD7095552747FD5095CE01CC
:105A00000E948525CE010E94C825CE01B701A801BC
:105A100096010E94EA25DF91CF911F910F91FF908F
:105A2000EF90DF90CF90BF9008950F931F93CF9387
:105A3000DF938C01EB016881662329F0C8010E9485
:105A4000262C2196F8CFDF91CF911F910F910895C9
:105A50000F931F93CF93DF938C01EB01FE016491B1
:105A6000662329F0C8010E94262C2196F7CFDF91EA
:105A7000CF911F910F910895FC0184A5482F5527C0
:105A800047FD50951416150624F176A5671748F0C2
:105A9000272F30E0260F311D87A590E02817390702
:105AA0000CF06FE3671B262F332727FD3095C901C4
:105AB0009595879502A4F3A5E02DE80FF91F849131
:105AC00020FD869590E08F7090709C01241B350B13
:105AD000A901CA010895EF92FF920F931F93CF93EC
:105AE000DF937C018B01C0E0D0E0F8016081662388
:105AF00041F0C7010E943C2DC80FD91F0F5F1F4FF7
:105B0000F4CFCE01DF91CF911F910F91FF90EF90D5
:105B10000895EF92FF920F931F93CF93DF937C0131
:105B20008B01C0E0D0E0F8016491662341F0C70129
:105B30000E943C2DC80FD91F0F5F1F4FF4CFCE011D
:105B4000DF91CF911F910F91FF90EF900895282F33
:105B5000FB0182859385622F0E94262C80E090E0D5
:105B60000895DC01FB01CB010196E4919C96EC9336
:105B70009C979C012F5F3F4FFC0184919D968C93D5
:105B80009D97C9010196F90124919E962C939E97A9
:105B9000FC0124919F962C939F9701969B969C9332
:105BA0008E939A970895DF93CF93CDB7DEB72E9754
:105BB0000FB6F894DEBF0FBECDBF27EA3DE23A87AD
:105BC00029879C878B8782E08C831E861D86CE0169
:105BD00001960E9439302E960FB6F894DEBF0FBEA4
:105BE000CDBFCF91DF910895DF93CF93CDB7DEB7CF
:105BF0009E01275F3F4F8D819E816F817885A9012E
:105C00000E94D32DCF91DF910895DF93CF93CDB72D
:105C1000DEB72E970FB6F894DEBF0FBECDBF27EAD2
:105C20003DE23A8729879C878B8782E08C831E869A
:105C30001D86CE0101960E9436322E960FB6F8943C
:105C4000DEBF0FBECDBFCF91DF910895DF93CF931D
:105C5000CDB7DEB79E01275F3F4F8D819E816F815B
:105C60007885A9010E94052ECF91DF9108953F927A
:105C70004F925F926F927F928F929F92AF92BF925C
:105C8000CF92DF92EF92FF920F931F93CF93DF9308
:105C90008C017B01EA010E94E724882309F4B6C045
:105CA000C80102960E94E724882309F4AFC0D801F6
:105CB00090964D915C91919792966D917C9193976E
:105CC0004115510519F46115710511F1F80184A10F
:105CD00083FF03C0CB01BA01AC01D70113968C91AD
:105CE000139782FF15C06C9F90016D9F300D7C9FB4
:105CF000300D1124240F351F220F331F16968D915E
:105D00009C911797820F931F17969C938E931697CB
:105D1000F80144885588C688D78884A1682F70E028
:105D200083FF03C0C60162012C013E01641875089F
:105D3000660C771C4398B3E075956795BA95E1F7C3
:105D40006770606FC8010E94C12333245201D701DC
:105D500013968C91139782FF13C016962D913C9148
:105D6000179783FF04C0F901C591D49103C0D901ED
:105D7000CD91DC912E5F3F4FF701378326830CC016
:105D8000C7010E94F72FEC01C7010E94F72F982E40
:105D90008824D070C829D929D80195968C919597D7
:105DA00081FF12C098968D919C919997C817D90739
:105DB00019F4332433940BC0332031F0C801B501FA
:105DC000A6010E941F243324CE010E94442308947C
:105DD000A108B108A114B10409F0B9CF611471048C
:105DE00051F0F701838182FF06C086819781860D7D
:105DF000971D978386830894C108D108C114D104E4
:105E000009F0A4CFC8010E94D425439AC8010E947A
:105E10008224DF91CF911F910F91FF90EF90DF903F
:105E2000CF90BF90AF909F908F907F906F905F903A
:105E30004F903F900895DF93CF93CDB7DEB72E9765
:105E40000FB6F894DEBF0FBECDBF1A8619861C862A
:105E50001B862DE02C831E861D8678876F83BE01EE
:105E60006F5F7F4F0E94372E2E960FB6F894DEBFDD
:105E70000FBECDBFCF91DF91089520E067FF02C034
:105E8000409A01C0409881E0982F9A95F1F7419A85
:105E9000982F9A95F1F7660F41988A95F1F718991E
:105EA0006F5F2F5F283051F7862F08950F931F9350
:105EB0008C0188B18C7F88B987B1836087B985B13F
:105EC000836085B9C80160E00E943D2FC80160E091
:105ED0000E943D2FC80160E00E943D2F1F910F914D
:105EE000089583B18695809581700895FF920F93F0
:105EF0001F938C010E943D2F88E08A95F1F7C8011D
:105F000060E00E943D2FF82EC80160E00E943D2F06
:105F10005F2D40E0282F30E0242B352BC9011F9145
:105F20000F91FF900895A0E0B0E0E9E9FFE20C9442
:105F3000B335EC01A880B980CA80DB80A114B1041C
:105F4000C104D10441F484E2A82E89EDB82E8BE57A
:105F5000C82E87E0D82EC601B5012DE133EF41E010
:105F600050E00E94903527EA31E440E050E00E9482
:105F70005E357B018C01C601B5012DE133EF41E0B7
:105F800050E00E949035CA01B9012CEE34EF4FEF7A
:105F90005FEF0E945E356E0D7F1D801F911F97FF82
:105FA00004C06150704080409048688379838A8340
:105FB0009B839B013F77C901CDB7DEB7EAE00C9424
:105FC000CF350E94932F089580E091E00E94932F97
:105FD0000895A0E0B0E08093000190930101A093A8
:105FE0000201B09303010895F8940C941836CF93EE
:105FF000DF93EC014B8140FF1AC046FF0AC04F7B84
:106000004B838E819F8101969F838E838A81282F67
:106010002BC042FF13C0E881F9818081282F3327EC
:1060200027FD30952115310529F440624B832FEF70
:106030003FEF1BC03196F983E88311C0EA85FB85E9
:10604000CE0109959C0197FF0AC09B812F5F3F4FAE
:1060500011F080E201C080E1892B8B83E8CF8E8133
:106060009F8101969F838E8330E0C901DF91CF919C
:1060700008950F931F938C01FC01838188608383B3
:10608000C8010E943632F8012381277F23831F91A4
:106090000F910895F0D0E39526C10CD013C1E3D041
:1060A00040F0DAD030F021F45F3F19F0CCC051114C
:1060B0004EC1CFC029D198F39923C9F35523B1F329
:1060C000951B550BBB27AA2762177307840738F067
:1060D0009F5F5F4F220F331F441FAA1FA9F333D0C6
:1060E0000E2E3AF0E0E830D091505040E695001C7A
:1060F000CAF729D0FE2F27D0660F771F881FBB1F36
:10610000261737074807AB07B0E809F0BB0B802D0F
:10611000BF01FF2793585F4F2AF09E3F510568F05B
:1061200092C015C15F3FECF3983EDCF386957795FE
:106130006795B795F7959F5FC9F7880F911D96955D
:10614000879597F90895E1E0660F771F881FBB1FB9
:10615000621773078407BA0720F0621B730B840B66
:10616000BA0BEE1F88F7E095089504D06894B1113A
:10617000EEC00895D1D088F09F5790F0B92F99279D
:10618000B751A0F0D1F0660F771F881F991F1AF042
:10619000BA95C9F712C0B13081F0D8D0B1E00895F6
:1061A000D5C0672F782F8827B85F39F0B93FCCF377
:1061B000869577956795B395D9F73EF49095809538
:1061C000709561957F4F8F4F9F4F0895E89409C058
:1061D00097FB3EF490958095709561957F4F8F4F1A
:1061E0009F4F9923A9F0F92F96E9BB279395F69530
:1061F000879577956795B795F111F8CFFAF4BB0FAE
:1062000011F460FF1BC06F5F7F4F8F4F9F4F16C011
:10621000882311F096E911C0772321F09EE8872F9B
:10622000762F05C0662371F096E8862F70E060E057
:106230002AF09A95660F771F881FDAF7880F9695D0
:10624000879597F9089597F99F6780E870E060E077
:1062500008959FEF80EC089500240A9416161706FF
:1062600018060906089500240A9412161306140647
:1062700005060895EECF50D0E8F3E894E0E0BB27A0
:106280009F57F0F02AED3FE049EC06C0EE0FBB0F40
:10629000661F771F881F28F0B23A620773078407CA
:1062A00028F0B25A620B730B840BE3959A9572F740
:1062B000803830F49A95BB0F661F771F881FD2F77E
:1062C0009048B3C3092E0394000C11F4882352F0B4
:1062D000BB0F40F4BF2B11F460FF04C06F5F7F4F12
:1062E0008F4F9F4F0895EF93E0FF06C0A2EA2AED7B
:1062F0003FE049EC5FEB44D3E5DF0F90039401FCF2
:106300009058E8E6F0E09DC357FD9058440F551FA4
:1063100059F05F3F71F04795880F97FB991F61F027
:106320009F3F79F087950895121613061406551F9E
:10633000F2CF4695F1DF08C0161617061806991F0A
:10634000F1CF86957105610508940895E894BB27FF
:1063500066277727CB0197F908950BD0B3CF7CDF61
:1063600028F081DF18F0952309F06DCF72CF11244A
:10637000EECFCADFA0F3959FD1F3950F50E0551FE4
:10638000629FF001729FBB27F00DB11D639FAA278A
:10639000F00DB11DAA1F649F6627B00DA11D661FD9
:1063A000829F2227B00DA11D621F739FB00DA11DFA
:1063B000621F839FA00D611D221F749F3327A00DB4
:1063C000611D231F849F600D211D822F762F6A2F50
:1063D00011249F5750408AF0E1F088234AF0EE0FD5
:1063E000FF1FBB1F661F771F881F91505040A9F7E2
:1063F0009E3F510570F027CFAACF5F3FECF3983E48
:10640000DCF3869577956795B795F795E7959F5F48
:10641000C1F7FE2B880F911D9695879597F90895E2
:106420009F9329DF0F9007FCEE5F5DCFDF93D92F9D
:1064300022DFE695D7952AED3FE049E45FE3B33AE2
:106440006207730784079507D7952AF0A2EA49ECFB
:10645000906896D237DFE6E8F0E0F3D2DD0F0BF07C
:1064600001D3DD0F0BF49058DF910895ABE0B0E05D
:10647000ECE3F2E30C94AB353C012B015A01FC0137
:1064800017821682838181FD03C06FEF7FEFC6C143
:106490009AE0892E1E010894211C311CF3012381EE
:1064A000F20123FD859123FF81912F01882309F4B7
:1064B000B2C1853239F423FD859123FF81912F01EB
:1064C000853229F490E0B3010E942934E7CF982F58
:1064D000FF24EE249924FFE1FF15D0F09B3269F0F0
:1064E0009C3228F4903259F0933291F40EC09D32D0
:1064F00049F0903369F441E024C052E0F52A84E089
:10650000F82A28C098E0F92A25C0E0E1FE2A22C036
:10651000F7FC29C0892F80538A3070F4F6FE05C03D
:10652000989C902C1124980E15C0E89CE02C112406
:10653000E80EF0E2FF2A0EC09E3229F4F6FC6BC191
:1065400040E4F42A07C09C3619F450E8F52A02C04A
:10655000983649F4F20123FD959123FF91912F0183
:10656000992309F0B8CF892F8554833018F08052D1
:10657000833038F444E050E0A40EB51E5FE3598345
:106580000FC0933631F0933779F0933509F056C048
:1065900020C0F5018081898342E050E0A40EB51E41
:1065A000610101E010E012C0F501C080D180F6FC6D
:1065B00003C06FEF7FEF02C0692D70E042E050E052
:1065C000A40EB51EC6010E941E348C015FE7F522A1
:1065D00014C0F501C080D180F6FC03C06FEF7FEFDF
:1065E00002C0692D70E042E050E0A40EB51EC60165
:1065F0000E9413348C0150E8F52AF3FE07C01AC03C
:1066000080E290E0B3010E942934EA948E2D90E05C
:1066100008171907A8F30EC0F601F7FC8591F7FEDD
:1066200081916F0190E0B3010E942934E110EA9456
:10663000015010400115110579F7EAC0943611F0A8
:10664000993669F5F7FE08C0F50120813181428154
:10665000538184E090E00AC0F501808191819C0122
:10666000442737FD4095542F82E090E0A80EB91ED4
:106670009FE6F92257FF09C0509540953095219526
:106680003F4F4F4F5F4FE0E8FE2ACA01B901A10119
:106690002AE030E00E945534D82ED21840C09537F9
:1066A00029F41F2D1F7E2AE030E01DC01F2D197F09
:1066B0009F3661F0903720F4983509F0ACC00FC0D8
:1066C000903739F0983709F0A6C004C028E030E0D0
:1066D0000AC0106114FD146020E130E004C014FD14
:1066E000166020E132E017FF08C0F501608171817A
:1066F0008281938144E050E008C0F501808191815E
:10670000BC0180E090E042E050E0A40EB51EA10183
:106710000E945534D82ED2188FE7F82EF122F6FEBB
:106720000BC05EEFF522D91438F4F4FE07C0F2FC7A
:1067300005C08FEEF82202C01D2D01C0192DF4FEF8
:106740000DC0FE01ED0DF11D8081803319F499EE2D
:10675000F92208C01F5FF2FE05C003C08F2D8678A6
:1067600009F01F5F0F2DF3FC14C0F0FE0FC01E15C3
:1067700010F09D2C0BC09D2C9E0C911A1E2D06C056
:1067800080E290E0B3010E9429341F5F1E15C0F320
:1067900004C01E1510F4E11A01C0EE2404FF0FC05E
:1067A00080E390E0B3010E94293402FF1DC001FD87
:1067B00003C088E790E00EC088E590E00BC0802F12
:1067C000867891F001FF02C08BE201C080E2F7FC05
:1067D0008DE290E0B3010E94293406C080E390E08E
:1067E000B3010E9429349A94D914C0F3DA94F101C8
:1067F000ED0DF11D808190E0B3010E942934DD2070
:10680000A9F706C080E290E0B3010E942934EA941F
:10681000EE20C1F743CEF30166817781CB012B9641
:10682000E2E10C94C735FC01059061507040011005
:10683000D8F7809590958E0F9F1F0895FC016150A9
:10684000704001900110D8F7809590958E0F9F1F92
:1068500008950F931F93CF93DF938C01EB018B81EE
:1068600081FF1BC082FF0DC02E813F818C819D81E5
:106870002817390764F4E881F9810193F983E883E3
:1068800006C0E885F985802F0995892B31F48E8122
:106890009F8101969F838E8302C00FEF1FEFC80177
:1068A000DF91CF911F910F910895FA01AA27283007
:1068B00051F1203181F1E8946F936E7F6E5F7F4FCD
:1068C0008F4F9F4FAF4FB1E03ED0B4E03CD0670F49
:1068D000781F891F9A1FA11D680F791F8A1F911D9C
:1068E000A11D6A0F711D811D911DA11D20D009F4EC
:1068F00068943F912AE0269F11243019305D31932E
:10690000DEF6CF010895462F4770405D4193B3E016
:106910000FD0C9F7F6CF462F4F70405D4A3318F0BD
:10692000495D31FD4052419302D0A9F7EACFB4E06E
:10693000A6959795879577956795BA95C9F7009726
:106940006105710508959B01AC010A2E06945795C7
:10695000479537952795BA95C9F7620F731F841F1E
:10696000951FA01D089578DC30F07DDC20F031F417
:106970009F3F11F41EF46DCC0EF4E095E7FB63CC61
:10698000E92FC2DC80F3BA17620773078407950703
:1069900018F071F49EF5DACC0EF4E0950B2EBA2FB8
:1069A000A02D0B01B90190010C01CA01A001112415
:1069B000FF27591B99F0593F50F4503E68F11A16C1
:1069C000F040A22F232F342F4427585FF3CF469552
:1069D00037952795A795F0405395C9F77EF41F1674
:1069E000BA0B620B730B840BBAF09150A1F0FF0F3E
:1069F000BB1F661F771F881FC2F70EC0BA0F621F2A
:106A0000731F841F48F4879577956795B795F79519
:106A10009E3F08F0B3CF9395880F08F09927EE0FAB
:106A20009795879508959F3F31F0915020F4879571
:106A300077956795B795880F911D9695879597F9E6
:106A400008959F938F937F936F93FF93EF939B0191
:106A5000AC0183DCEF91FF910CD02F913F914F91CE
:106A60005F917BCC9B01AC0160E070E080E89FE32C
:106A700014CBDF93CF931F930F93FF92EF92DF928C
:106A80007B018C01689405C0DA2EEF0172DCFE01F7
:106A9000E894A5912591359145915591AEF3EF017B
:106AA0006FDFFE019701A801DA9479F7DF90EF908C
:106AB000FF900F911F91CF91DF910895629FD001B8
:106AC000739FF001829FE00DF11D649FE00DF11DA9
:106AD000929FF00D839FF00D749FF00D659FF00D58
:106AE0009927729FB00DE11DF91F639FB00DE11D45
:106AF000F91FBD01CF011124089597FB092E072628
:106B00000AD077FD04D05ED006D000201AF470952C
:106B100061957F4F0895F6F7909581959F4F089561
:106B200097FB092E05260ED057FD04D05FD00AD062
:106B3000001C38F450954095309521953F4F4F4FAC
:106B40005F4F0895F6F790958095709561957F4F0A
:106B50008F4F9F4F08952F923F924F925F926F9267
:106B60007F928F929F92AF92BF92CF92DF92EF92DD
:106B7000FF920F931F93CF93DF93CDB7DEB7CA1B5E
:106B8000DB0B0FB6F894DEBF0FBECDBF09942A8889
:106B9000398848885F846E847D848C849B84AA8431
:106BA000B984C884DF80EE80FD800C811B81AA81BE
:106BB000B981CE0FD11D0FB6F894DEBF0FBECDBF89
:106BC000ED010895AA1BBB1B51E107C0AA1FBB1F03
:106BD000A617B70710F0A61BB70B881F991F5A9569
:106BE000A9F780959095BC01CD010895A1E21A2ED8
:106BF000AA1BBB1BFD010DC0AA1FBB1FEE1FFF1F61
:106C0000A217B307E407F50720F0A21BB30BE40BB0
:106C1000F50B661F771F881F991F1A9469F76095F7
:106C20007095809590959B01AC01BD01CF010895B1
:046C3000F894FFCF06
:046C3400010000005B
:00000001FF
